:020000040000FA
:100000000C9468190C9490190C9490190C94422C2F
:100010000C9490190C9490190C9490190C949019BC
:100020000C9490190C9490190C9490190C949019AC
:100030000C9490190C9490190C9490190C9490199C
:100040000C94F82B0C9490190C94C62B0C94A02BA8
:100050000C9490190C94192D0C9490190C949019DF
:100060000C9490190C94901900000000000F1DC210
:100070000800054442080003845FBF000FE44410F9
:10008000000115451000054CC97F8009244F9000E0
:1000900007C4C11000054D413F00055443810007CE
:1000A000C44D02000544411400055541080007C82D
:1000B0008104000000000000000000000001083F73
:1000C000FE001FFF810000004002000007FE0FF845
:1000D000000402080800040208880007FE088800DF
:1000E0000402088800040208880007FE088800044B
:1000F00002094800040202300007FE040C0004025A
:1001000018040000000000000000000000011000C2
:1001100080001FFF80800001103FFF0000400408A6
:100120000007FC040800044404100004440210000A
:1001300004440220001FFF812000004000C0000096
:10014000A00130000110020800060C0C0700180383
:10015000B0020000000000000000000000004000AD
:10016000800000400080000FFF3FFF0008410408AE
:100170000008410408000841041000084102100072
:100180000FFF0220000841012000004000C00000D5
:1001900040013000004002080000400C0700004011
:1001A000300200000000000000000000001FDF100F
:1001B000200002120C20000224042000047F802072
:1001C000000424B820000FA488500014BF885000F9
:1001D00004A488500004A488480004BF8888000450
:1001E000A48A880007A48C84000444890700008145
:1001F000860200000000000000000000000FF00474
:1002000091000440025200047F905400045088FF83
:100210000007D08481000451008100044901FF00DF
:1002200007CA0281000444048100044A1CFF00073D
:10023000EA0481000C510481000061C48500004083
:100240008082000000000000000000000007FF8026
:100250002000008407FF00008404010000840401E2
:100260000000840401000FFFC7FF000084040000A9
:100270000084040000008405FF00008405010001E3
:10028000040901000104090100020411FF00040433
:1002900001010000000000000000000000008204D6
:1002A000FF00004402010007FF9021000010102110
:1002B00000001017FD0000101021000FFFD061009A
:1002C000001010A1000028112100002812210000B8
:1002D00044142100008210A1000301D045000C004D
:1002E0009002000000000000000000000008441020
:1002F000FE00042810920005FF22920000103C929C
:100300000000100892001CFE109200041020FE0055
:1003100004103E920005FF80920004100092000538
:10032000100E92000610309200041000FE00001023
:100330000082000000000000000000000007DF88CD
:1003400040000A24104000114210FE0004002282E6
:100350000002FF3D020008010A420009F9103200C4
:10036000090920120009F93E0200090900020009EA
:10037000090E020009F930220008050014000802E5
:10038000000800000000000000000000000FC3F1A2
:10039000E0000FE3F1F8000C70C19E000C30C18644
:1003A000000C30C183000C30C183000C60C183009D
:1003B0000C60C183000FC0C183000FC0C186000C58
:1003C00000C186000C00C198000C03F1F8000C037A
:1003D000F1E0000000000000000000000000200824
:1003E00020000FFF09FC00002008000000203E88CC
:1003F0000003FE08500002020BFE0003FE0C40004A
:10040000020218400003FE2BFE000202084800030F
:10041000FE088800020208500002022830001FFF78
:1004200091CC0000000000000104047C000088045E
:1004300044000FFF3F4400002004440000200C440F
:100440000000200E44001FFF9544000020144400CB
:10045000005024440000500444000088044500017A
:100460000404850006038503001801040000000051
:1004700000000000000000000000000000047E21D9
:10048000FC0004421104001F7E090400044221FC08
:10049000000542110400067E1104000C0005FC005A
:1004A00015FF880000040813FE00044832520004BF
:1004B0004F125200044812520014A8125200091F91
:1004C00097FF000000000000000000000002103D47
:1004D000FC000210250400041025040005FFBDFCEB
:1004E000000C102520000C38252000143825FE00B3
:1004F00004543D20000454251000049225100005EA
:1005000011A5090006113D450004102583000410C3
:10051000010100000000000000000000001FC810E2
:100520002000124A0C20001AC9042000174800209D
:10053000001FFFB8200002080850001FC808500024
:10054000020808500003C80848001E14088800016B
:10055000540A880015220C84001443890700008186
:10056000060200000000000002FE01000002823FBF
:10057000FF00048202000004FE0200000C1004FCD4
:1005800000141004080005FF8C1000041014100063
:10059000043825FF00043404100004520410000441
:1005A0009184100005100450000410042000000085
:1005B0000000000000000000000000000002030036
:1005C00010001FDC3EFE000890021200051004FF20
:1005D000001FDF84120002120CFE001FD202100066
:1005E000021222FE000A921410000A521410001285
:1005F000220DFF0002220810000A4214100004021B
:1006000023FF00000000000000000000000F78BC85
:1006100020000948A45000094AA85000094AA888A7
:1006200000094AB104001FFEAAFB00094AA42000E9
:10063000094AA42000094AA7FE00094AB42000097B
:1006400048A924000B48A22200088AA4A20011197C
:10065000204000000000000000000000000020001A
:100660008000005001FC0000880104000104030820
:100670000006FB0490000800C0600007DF01800056
:10068000045106000004511BFE0004510202000741
:10069000D90202000456020200001003FE000010FE
:1006A000020200000000000000000000000208201C
:1006B0009000027F9890001F8009FF000222011025
:1006C0000006218B100007628DFE000AA2091000AF
:1006D0000A14111000121431FE0002081110000259
:1006E000141110000222111000024391FF00028138
:1006F00011000000000000000000000000100700D2
:10070000000008F83FFE0004802002000080200264
:100710000000BE23E2001C8222220004A422220048
:1007200004942222000488222200049423E200057B
:100730002220020005422002000A003FFE0011FFB5
:10074000A002000000000000000000000001041FE3
:10075000FC0000880080000FFF0080000020008067
:1007600000002000800000203FFF001FFF8080006D
:100770000020008000005000800000500080000039
:1007800088008000010400800006038280001801B8
:10079000010000000000000009FF00400004203FAD
:1007A000FF00042000000000FE0000001C420FFCBF
:1007B00000044200000007FF80000004000FFC005E
:1007C00004FF000000048100000005810FFC00060A
:1007D0008108040004FF08040000810FFC000000F1
:1007E00000000000000000000000000000004000C9
:1007F00080001FFF9FFC0000400410000FFF02203C
:100800000000003FFF000FFE00000008420FF8004C
:1008100008420808000FFE08080008020FF8000848
:1008200000080800080008080008000FF800100081
:100830000808000000000000000000000007FE0F94
:10084000F8000402000000040200000007FE00009F
:100850000004023FFE00040200800007FE0080004A
:10086000009004900008910C880006931086000206
:1008700094208200009000800000900280001FFF02
:1008800081000000000000000000000000041012C1
:10089000020005FF9FD20005009212001E28A2123E
:1008A0000004443FF200048202120006000212001B
:1008B0000CFE1FD200141012520004101242000449
:1008C00010134200041012820015FF820A00080073
:1008D00002040000000000000000000000002000F2
:1008E000000000203E04001FFFA204001000A2FF31
:1008F0000000012204000FFE22040000403E4400DC
:1009000000402224000440222400047C220400042D
:10091000402204000A403E0400094022240010FF47
:100920008014000000000800000000000010FE0815
:10093000200008820BFF0004820A010010FE3C51D7
:10094000000882088800088209040002FE0C0000EA
:10095000040019FC0009FF282000192908200009BB
:1009600029082000092908200009292BFF000BFF76
:10097000900000000000000000000000001F7F90B9
:10098000F80001080888000A10088800047F0107A1
:10099000001FC13A0000054909FC00044908840011
:1009A0000449088800044908480004490850000424
:1009B000490A200004160C5800142189870008C039
:1009C00086020000000000000FFFFFFFFFF03FFF66
:1009D000FFFFFFFC7FFFFFFFFFFE7FFFFFFFFFFE2C
:1009E000F0000000000FF0000000000FF000000019
:1009F000000FF1FFFFFFFF8FF1FFFFFFFF8FF1FF00
:100A0000FFFFFF8FF1FFFFFFFF8FF1FFFFFFFF8F62
:100A1000F1FFFFFFFF8FF1FFFFFFFF8FF1FFFFFFF0
:100A2000FF8FF1FFFFFFFF8FF1FFFFFFFF8FF1FF50
:100A3000FFFFFF8FF1FFFFFFFF8FF1FFFF03FF8F2E
:100A4000F1FFFF03FF8FF1FFFF03FF8FF1FFFFFFB8
:100A5000F18FF1FFFFFFE18FF1FFFFFFC78FF1FF84
:100A6000FFFF8F8FF1FFFFFF0F8FF1FFFFFF8F8FD2
:100A7000F1FFFFFFC78FF1FFFFFFE18FF1FFFFFFE6
:100A8000F18FF1FFFFFFFF8FF1FFFFFFFF8FF000FE
:100A90000000000FF0000000000FF0000000000F49
:100AA000F1FFFFFFFF8FF1111FFFFF8FF1111FFFFC
:100AB000FF8FF1111FFFFF8FF1FFFFFFFF8FF0008E
:100AC0000000000FF0000000000FF0000000000F19
:100AD0007FFFFFFFFFFE7FFFFFFFFFFE3FFFFFFFE8
:100AE000FFFC0FFFFFFFFFF00FFFFFFFFFF03FFFD7
:100AF000FFFFFFFC7FFFFFFFFFFE7FFFFFFFFFFE0B
:100B0000FFFFFFFFFFFFFFFFFFFFFFFFFFFFFFFFF5
:100B1000FFFFFFFFFFFFFFFFFFFFFFFFFFFFFFFFE5
:100B2000FFFFFFFFFFFFFFFFFFFFFFFFFFFFFFFFD5
:100B3000FFFFFFFFFFFFFFFFFFFFFFFFFFFFFFC7FD
:100B4000001FC00FFFC7001FC00C1FC7001FC00C35
:100B50001FC71FFFC7FC0FC71FFFC7FC4FC71FFFE3
:100B6000C7FC4FC71FFFC7FC47C71FFFC7FC67C7AE
:100B70001C01C01C63C71C01C01C73C71C01C01C26
:100B800071C71F8FC7FC79C71F8FC7FC78C71F8F1E
:100B9000C7FC7C071F8FC7FC7C07000FC00C7E07BB
:100BA000000FC00FFFFF000FC00FFFFFFFFFFFFF91
:100BB000FFFFFFFFFFFFFFFFFFFFFFFFFFFFFFFF45
:100BC000FFFFFFFFFFFFFFFFFFFFFFFFFFFFFFFF35
:100BD000FFFFFFFFFFFFFFFFFFFFFFFFFFFFFFFF25
:100BE000FFFFFFFFFFFFFFFFFFFFFFFFFFFFFFFF15
:100BF0007FFFFFFFFFFE7FFFFFFFFFFE3FFFFFFFC7
:100C0000FFFC0FFFFFFFFFF00FFFFFFFFFF03FFFB5
:100C1000FFFFFFFC7FFFFFFFFFFE7FFFFFFFFFFEE9
:100C2000FFFFFFFFFFFFFFFFFFFFFFFFFFFFFFFFD4
:100C3000FFFFFFFFFC7FFFFFFFFFFC7FFFFFFFFFCA
:100C4000FC7FFFFFFFFFFC7FFFFFFFFFFC7FFFFF3D
:100C5000FFFFFC7FFFFFFFFFFC7FFFFFFFFFFC7F2D
:100C6000FFFFFE00000001FFFE00000001FFFE008C
:100C7000000001FFFE3FFC7FF1FFFE3FFC7FF1FF24
:100C8000FE3FFC7FF1FFFE3FFC7FF1FFFE3FFC7F5C
:100C9000F1FFFE3FFC7FF1FFFE3FFC7FF1FFFE3FD7
:100CA000FC7FF1FFFE3FFC7FF1FFFE000000007FB4
:100CB000FE000000007FFE000000007FFE3FFC7F82
:100CC000FFFFFFFFFC7FFFFFFFFFFC7FFFFFFFFF3A
:100CD000FC7FFFFFFFFFFC7FFFFFFFFFFC7FFFFFAD
:100CE000FFFFFC7FFFFFFFFFFC7FFFFFFFFFFC7F9D
:100CF000FFFFFFFFFC7FFFFFFFFFFC7FFFFFFFFF0A
:100D0000FCFFFFFFFFFFFFFFFFFFFFFFFFFFFFFFF6
:100D10007FFFFFFFFFFE7FFFFFFFFFFE3FFFFFFFA5
:100D2000FFFC0FFFFFFFFFF00FFFFFFFFFF03FFF94
:100D3000FFFFFFFC7FFFFFFFFFFE7FFFC003FFFE03
:100D4000FFFF0000FFFFFFFC00003FFFFFF000007F
:100D50000FFFFFC0000003FFFFC0000001FFFF0006
:100D6000000000FFFF000000007FFE000000007F89
:100D7000FC000000003FFC000000203FF8000000E5
:100D8000701FF8000000F81FF0000001F80FF000DD
:100D90000003F00FF0000007E00FF000000FC00F9D
:100DA000E000001F8007E001803F0007E003C07EF5
:100DB0000007E007E0FC0007E003F1F80007E001AE
:100DC000FFF00007E000FFE00007E0007FC0000741
:100DD000F0003F80000FF0001F00000FF0000E0039
:100DE000000FF0000400000FF8000000001FF800E2
:100DF0000000001FFC000000003FFC000000003F5E
:100E0000FF000000007FFF00000000FFFF800000E7
:100E100001FFFFC0000003FFFFF0000007FFFFF02D
:100E200000000FFFFFFC00003FFFFFFF0000FFFF7F
:100E30007FFFF00FFFFE7FFFFFFFFFFE3FFFFFFF83
:100E4000FFFC0FFFFFFFFFF00FFFFFFFFFF03FFF73
:100E5000FFFFFFFC7FFFFFFFFFFE7FFFC001FFFEE4
:100E6000FFFF0000FFFFFFFC00001FFFFFF000007E
:100E70000FFFFFE0000003FFFFC0000001FFFF8045
:100E8000000000FFFF000000007FFE000000007F68
:100E9000FE000000003FFC008000801FF801C0033E
:100EA000C01FF803E003E01FF803F00FE00FF001AC
:100EB000F80FC007F000FC1F8007F0007E7F0007DE
:100EC000E0003FFE0007E0001FFC0007E0000FF815
:100ED0000007E00007F00007E00007F00007E0006F
:100EE0001FF80007E0001FFC0007E0007FFE00077E
:100EF000F0007E3F0007F001FC1F8007F001F80FB3
:100F0000C00FF803F007E00FF803E003E01FF8015B
:100F1000C001801FFE008000803FFE000000003FF7
:100F2000FF000000007FFF000000007FFF80000046
:100F300000FFFFC0000001FFFFF0000007FFFFF807
:100F400000000FFFFFFC00003FFFFFFF8000FFFFDE
:100F50007FFFF007FFFE7FFFFFFFFFFE3FFFFFFF6A
:100F6000FFFC0FFFFFFFFFF00FFFFFFFFFF03FFF52
:100F7000FFFFFFFC7FFFFFFFFFFE7FFFF00FFFFE85
:100F8000FFFFF00FFFFFFFFFE007FFBFFFFFC3C33F
:100F9000FF1FFFFF87E1FE0FFFFF0FF0FC1FFFFEAB
:100FA0001FF8783FFFFC3FFCF07FFFF87FFFE0FF7A
:100FB000FFF0FFFFC1FFFFE1FFFF83FFFFE3FFFF44
:100FC00007FFFFE3FFFE07FFFFE3FFFC07FFFFE371
:100FD000FFF807FFFFE3FFF047FFFFE3FFE0C7FF76
:100FE000FFE3FFC1C7FFFFE3FF83C7FFFFE3FF0787
:100FF000C7FFFFE3FE0FC7FFFFE3FC1FC7FFFFE3D1
:10100000F83FC7FFFFE3F07FC7FFFFE3E0FFC7FF45
:10101000FFE3C1FFC7FFFFE783FFC7FFFFEF07FF46
:10102000C7FFFFFE0FFFC1FFFFFC1FFFE0FFFFF840
:101030003FFFF87FFFF07FFFFC3FFFE00000003F35
:10104000FFC00000003FFF800000003FFF07FFFFE0
:10105000FFFFFE0FC003FFFFFC1FC003FFFFFE3FAB
:10106000E007FFFFFF7FE007FFFFFFFFF81FFFFF25
:101070007FFFF81FFFFE7FFFFFFFFFFE3FFFFFFF29
:10108000FFFC0FFFFFFFFFF00FFFFFFFFFF03FFF31
:10109000FFFFFFFC7FFFFFFFFFFE7FFFFFFFFFFE65
:1010A000F0000000000FF0000000000FF000000052
:1010B000000FF1FFFFFFFF8FF1FFFFF8888FF1FFB7
:1010C000FFF8888FF1FFFFF8888FF1FFFFFFFF8F98
:1010D000F0000000000FF0000000000FF000000022
:1010E000000FF1FFFFFFFF8FF10DDDFE4A8FF10AC8
:1010F000AAFFCD8FF10888FE5F8FF11AAAFFFF8F3C
:10110000F1FFFFFFFF8FF1FFFFFFFF8FF1FFFF00F8
:10111000008FF10C017FFF8FF16FFF46318FF16C73
:101120003F56B78FF11FFF56B78FF1FFFF46318F44
:10113000F1FFFF77B58FF1FFFF77B58FF10C0177E6
:10114000B58FF16FFF46318FF16C3F7FFF8FF11F3D
:10115000FF00008FF1FFFFFFFF8FF1FFFFFFFF8F09
:10116000F1FFFFFFFF8FF100002AA48FF10000556F
:10117000228FF1E0002AA48FF1FFFFFFFF8FF00024
:101180000000000FF0000000000FF0000000000F52
:101190007FFFFFFFFFFE7FFFFFFFFFFE3FFFFFFF21
:1011A000FFFC0FFFFFFFFFF00FFFFFFFFFF03FFF10
:1011B000FFFFFFFC7FFFFFFFFFFE7FFFFFFFFFFE44
:1011C000F0000000000FF0000000000FF000000031
:1011D000000FF1FFFFFFFF8FF1FFFFF8888FF1FF96
:1011E000FFF8888FF1FFFFF8888FF1FFFFFFFF8F77
:1011F000F0000000000FF0000000000FF000000001
:10120000000FF1FFFFFFFF8FF1FFFFFFFF8FF1FFE7
:10121000FFFFFF8FF1FFFFFFFF8FF1FFFFFFFF8F4A
:10122000F180F01F018FF180F01F018FF19CF39F7F
:10123000F98FF19CF39FF98FF19CF39FF98FF19C4B
:10124000F39FF98FF180F01C018FF180F01C018F6A
:10125000F1FCFF9CF98FF1FCFF9CF98FF1FCFF9CE6
:10126000F98FF1FCFF9CF98FF100E01C018FF10078
:10127000E01C018FF1FFFFFFFF8FF1FFFFFFFF8FEA
:10128000F1FFFFFFFF8FF1FFFFFFFF8FF1FFFFFF78
:10129000FF8FF1FFFFFFFF8FF1FFFFFFFF8FF000D8
:1012A0000000000FF0000000000FF0000000000F31
:1012B0007FFFFFFFFFFE7FFFFFFFFFFE3FFFFFFF00
:1012C000FFFC0FFFFFFFFFF00FFFFFFFFFF03FFFEF
:1012D000FFFFFFFC7FFFFFFFFFFE7FFFFFFFFFFE23
:1012E000FFFFFFFFFFFFFDFFFFFFFFFFF8FFFFFF17
:1012F000FFFFF07FFFFFFFFFE03FFFFFFFFFF8FF73
:10130000FFFFFFFFF8FFFFFFFFFFF8FFFFFFFFFFFB
:10131000F8E7FFFFFFFFF8E7FFE1FFFFF8E3FF005B
:101320007FFFF8F3FE0C1FFFF8F3F87F0FFFF8F1D3
:10133000F0FFC7FFF8F9E3FFE3FFF8F8E7FFF1FF7D
:10134000F8FC47FFF8FFF8FE0FFFFCFFF8FF1FFF58
:10135000FFFFF8FF1FFFFFFFF8FE0FFFFFFFF8FE84
:1013600047FFFFFFF8FC63FFFFFFF8FCF0FFFFFF04
:10137000F8F8F87FFFFFF8F9FE1FFFFFF8F1FF070D
:10138000FFFFF8E3FFC1FFFFF8C7FFF01FFFF8C73B
:10139000FFFC07FFF8CFFFFFC7FFF8FFFFFFFFFFCE
:1013A000F8FFFFFFFFFFF8FFFFFFFFBFF8FFFFFFA2
:1013B000FF9FF8000000000FF80000000007F80091
:1013C0000000000FFFFFFFFFFF9FFFFFFFFFFFBFBA
:1013D0007FFFFFFFFFFE7FFFFFFFFFFE3FFFFFFFDF
:1013E000FFFC0FFFFFFFFFF00FFFFFFFFFF03FFFCE
:1013F000FFFFFFFC7FFFFFFFFFFE7FFFFFFFFFFE02
:10140000FFFFFFFFFFFFFDFFFFFFFFFFF8FFFFFFF5
:10141000FFFFF07FFFFFFFFFE03FFFFFFFFFF8FF51
:10142000FFFFFFFFF8FFFFFFFFFFF8FFFFFFFFFFDA
:10143000F8E7FFFFFFFFF8E7C00003FFF8E3C00095
:1014400003FFF8F3CFFFFFFFF8F3CFFFFFFFF8F143
:10145000CFFFFFFFF8F9CFFFFFFFF8F8CFFFFFFF47
:10146000F8FC4FFFFFFFF8FE0FFFFFFFF8FF0FFF35
:10147000FFFFF8FF0FFFFFFFF8FF8FFFFFFFF8FFF1
:10148000C7FFFFFFF8FFC3FFFFFFF8FFC0FFFFFF2D
:10149000F8FFC87FFFFFF8800E1FFFFFF8800F07DF
:1014A000FFFFF8FFFFC1FFFFF8FFFFF01FFFF8FF8E
:1014B000FFFC07FFF8FFFFFFC7FFF8FFFFFFFFFF7D
:1014C000F8FFFFFFFFFFF8FFFFFFFFBFF8FFFFFF81
:1014D000FF9FF8000000000FF80000000007F80070
:1014E0000000000FFFFFFFFFFF9FFFFFFFFFFFBF99
:1014F0007FFFFFFFFFFE7FFFFFFFFFFE3FFFFFFFBE
:10150000FFFC0FFFFFFFFFF00FFFFFFFFFF03FFFAC
:10151000FFFFFFFC7FFFFFFFFFFE7FFFFE3FFFFEA1
:10152000FFFFFE3FFFFFFFFFFE3FFFFFFFFFFE3F0E
:10153000FFFFFFFFFE3FFFFFFFFFBE3DFFFFFFFE80
:101540003E3C7FFFFFFC3E3C3FFFFFF83E3C1FFF61
:10155000FFF0FE3F0FFFFFE1FE3F87FFFFC3FE3FAF
:10156000C3FFFF87FE3FE1FFFF8FFE3FF1FFFF0F4D
:10157000FE3FF0FFFF1FFE3FF8FFFF1FFE3FF8FF9B
:10158000FE1FFE3FFC7FFE3FFE3FFC7FFE3FFE3F17
:10159000FC7FFE3FFE3FFC7FFE3FFE3FFC7FFE3FA9
:1015A000FFFFFC7FFE3FFFFFFC7FFE1FFFFFFC7F76
:1015B000FF1FFFFFF8FFFF1FFFFFF8FFFF0FFFFFF9
:1015C000F0FFFF8FFFFFF1FFFF87FFFFE1FFFFC38A
:1015D000FFFFC3FFFFE1FFFF87FFFFF0FFFF07FFF4
:1015E000FFF83FFC0FFFFFFC0FF03FFFFFFE000086
:1015F0007FFFFFFF8001FFFFFFFFF00FFFFFFFFFF7
:10160000FFFFFFFFFFFFFFFFFFFFFFFFFFFFFFFFEA
:101610007FFFFFFFFFFE7FFFFFFFFFFE3FFFFFFF9C
:10162000FFFC0FFFFFFFFFF00FFFFFFFFFF03FFF8B
:10163000FFFFFFFC7FFEFFFFFFFE7FFE7FFFFFFE41
:10164000FFFE3FFFFFFFFFFE1FFFFFFFFFFE0FFF3D
:10165000FFFFFFFE07FFFFFFFFFE03FFFFFFFFFE91
:1016600001FFFFFFFFFE01FFFFFFFFFC00FFFFFF89
:10167000FFF800FFFFFFFFF000FFFFFFFFE0007F2C
:10168000FFFFFFE0007FFFFFFFC0007FFFFFFF8045
:10169000007FFFFFFF00007EFFFFFF00007E7FFF57
:1016A000FE0000FE3FFFFC0000FF1FFFFC0000FEED
:1016B0000FFFF80001FE07FFF80001FE03FFF00036
:1016C00003FC01FFF00007FC01FFF0000FF801FF31
:1016D000F0001FF000FFF0001FF000FFF0003FE0FF
:1016E000007FF8007FC0007FF800FF80007FFC00D3
:1016F000FF00007FFC01FF00007FFE01FE00007F75
:10170000FE03FC00007FFF03F80000FFFF83F800EA
:1017100000FFFFC7F80000FFFFE3F00001FFFFF349
:10172000F00003FFFFFFF00007FFFFFFFFFFFFFFD9
:101730007FFFFFFFFFFE7FFFFFFFFFFE3FFFFFFF7B
:10174000FFFC0FFFFFFFFFF00FFFFFFFFFF03FFF6A
:10175000FFFFFFFC7FFFFFFFFFFE7FFFFFC1FFFEDC
:10176000FFFFFF01FFFFFFFFFC01FFFFFFFFF00195
:10177000FFFFFFFFC001FFFFFFFF0007FFFFFFFCB0
:10178000001FFFFFFFF0007F9FFFFFE001FE0FFF44
:10179000FFC007F807FFFFC01FE007FFFFC07F8003
:1017A00007FFFFE1FE001FFFFFFFF8003FFFFFFF05
:1017B000E001FFFFFFFF8003FFFFFFFE000FFFFFC1
:1017C000FFF8003FFFFFFFE000FE0FFFFFC003FC3C
:1017D00007FFFFC00FE007FFFFC03FC007FFFFC0CC
:1017E000FE000FFFFFFFFC003FFFFFFFE0007FFF59
:1017F000FFFFC003FFFFFFFF0001FFFFFFFE00012F
:10180000FFFFFFFE0000FFFFFFFE0001FFFFFFFFE5
:101810000001FFFFFFFFFFFFFFFFFFFFFFFFFFFFD5
:10182000FFFFFFFFFFFFFFFFFFFFFFFFFFFFFFFFC8
:10183000FFFFFFFFE00FFFFFFFFFC007FFFFFFFFFE
:101840008007FFFFFFFF8007FFFFFFFFC00FFFFFC5
:101850007FFFE01FFFFE7FFFFFFFFFFE3FFFFFFF59
:10186000FFFC0FFFFFFFFFF00FFFFFFFFFF03FFF49
:10187000FFFFFFFC7FFFFFFFFFFE7FFFFFFFFFFE7D
:10188000F00000001FFFF00000000FFFF00000005C
:1018900007FFF1C00FF8C3FFF1C00FF8E1FFF1C07F
:1018A0000FF8F0FFF1C00FF8F87FF1C00FF8FC3F20
:1018B000F1C00FF8FE1FF1C00000FF0FF1C00000E3
:1018C000FF8FF1C00000FF8FF1FFFFFFFF8FF1FFDF
:1018D000FFFFFF8FF1FFFFFFFF8FF1FFFFFFFF8F84
:1018E000F1FFFFFFFF8FF1FFFFFFFF8FF1FFFFFF12
:1018F000FF8FF1FFFFFFFF8FF1FFFFFFFF8FF1C0B1
:101900000000038FF1C00000038FF1C00000038FBF
:10191000F1C7FFFFE38FF1C7FFFFE38FF1C60000C0
:10192000E38FF1C60000E38FF1C60000E38FF1C73B
:10193000FFFFE38FF1C7FFFFE38FF1C60000E38FE6
:10194000F1C60000E38FF1C60000E38FF1C7FFFF8F
:10195000E38FF1C7FFFFE38FF1C7FFFFE38FF000D5
:101960000000000FF0000000000FF0000000000F6A
:101970007FFFFFFFFFFE7FFFFFFFFFFE3FFFFFFF39
:10198000FFFC0FFFFFFFFFF00FFFFFFFFFF03FFF28
:10199000FFFFFFFC7FFFFFFFFFFE7FFFFFFFFFFE5C
:1019A000FFFFFFFFFFFFFFFFFFFFFFFFFFFFFFFF47
:1019B000FFFFFFFFFFFFFFFFFFFFFFFFFFFFFFFF37
:1019C000FFFFFFFFFFFFFFFFFFFFFFFFFE3FFFFFE8
:1019D000FFFFFE3FFFFFFFFFFE3FFFFFFFFFFE3F5A
:1019E000FFFFFFFFFE3FFFFFFFFFFE3FFFFFFFFF89
:1019F000FE3FFFFFFFFFFE3FFFFFFFFFFE3FFFFF3A
:101A0000FFFFFE3FFFFFFFFFFE3FFFFFFFF0000075
:101A10000FFFFFF000000FFFFFF000000FFFFFFFC0
:101A2000FFFFFFFFFFFFFE3FFFFFFFFFFE3FFFFF48
:101A3000FFFFFE3FFFFFFFFFFE3FFFFFFFFFFE3FF9
:101A4000FFFFFFFFFE3FFFFFFFFFFE3FFFFFFFFF28
:101A5000FE3FFFFFFFFFFE3FFFFFFFFFFFFFFFFF18
:101A6000FFFFFFFFFFFFFFFFFFFFFFFFFFFFFFFF86
:101A7000FFFFFFFFFFFFFFFFFFFFFFFFFFFFFFFF76
:101A8000FFFFFFFFFFFFFFFFFFFFFFFFFFFFFFFF66
:101A90007FFFFFFFFFFE7FFFFFFFFFFE3FFFFFFF18
:101AA000FFFC0FFFFFFFFFF00FFFFFFFFFF03FFE08
:101AB00000007FFC7FFE00007FFE7FFC00003FFEF9
:101AC000FFFC7FFE3FFFFFFC7FFE3FFFFFFC7FFE32
:101AD0003FFFFC000000001FF8000000000FF000B6
:101AE00000000007F1FFFFFFFFC7F1FFFFFFFFC787
:101AF000F1FFFFFFFFC7F00000000007F800000043
:101B0000000FFC000000001FFFFFFFFFFFFFFC7F36
:101B1000FFFFFE3FFC7FFFFFFE3FFC7FFFFFFE3F1E
:101B2000FC7F8FF8FE3FFC7F8FF8FE3FFC7F8FF835
:101B3000FE3FFC7F8FF8FE3FFC7F8FF8FE3FFC7F6F
:101B40008FF8FE3FFC7F8FF8FE3FFC7F8FF8FE3F53
:101B5000FC7F8FF8FE3FFC7F8FF8FE3FFC7F8FF805
:101B6000FE3FFC7F8FF8FE3FFC7F8FF8FE3FFC7F3F
:101B70008FF8FE3FFC7F8FF8FE3FFC7F8FF8FE3F23
:101B8000FC7F8FF8FE3FFC7FFFFFFE3FFC7FFFFFE7
:101B9000FE3FFC7FFFFFFE3FFC7FFFFFFE3FFC7F21
:101BA000FFFFFE3FFC3FFFFFFC3FFC000000003F4B
:101BB0007E000000007E7F00000000FE3FFFFFFF70
:101BC000FFFC0FFFFFFFFFF00FFFFFFFFFF03FFFE6
:101BD000FFFFFFFC7FFFFFFFFFFE7FFFFFFFFFFE1A
:101BE000FFFFFFFFFFFFFFFFFFFFFFFFFFFFFFFF05
:101BF000FFFFFFFFF007FFFFFFFF8000FFFFFFFE7B
:101C000000003FFFFFF807F00FFFFFF03FFE07FF68
:101C1000FFE0FFFF83FFFFC1FFFFE1FFFF87FFFF43
:101C2000F0FFFF0FFFFFF87FFF0FFFFFFC7FFE1F9E
:101C3000FFFFFC3FFE3FFFFFFE3FFC3FF3FBFE1FAD
:101C4000FC7FE1F0FF1FFC7FC0E07F1FF87F80403A
:101C50007F0FF8FF00003F8FF8FF00003F8FF8FF75
:101C600000001F8FF8FE00001F8FFFFE00001FFF07
:101C7000FFFE00001FFFFFFE00001FFFFFFF000030
:101C80001FFFFFFF00003FFFFFFF00003FFFFFFFC0
:101C900080007FFFFFFF80007FFFFFFFC000FFFF8E
:101CA000FFFFF003FFFFFFFFFC0FFFFFFFFFFFFF42
:101CB000FFFFFFFFFFFFFFFFFFFFFFFFFFFFFFFF34
:101CC000FFFFFFFFFFFFFFFFFFFFFFFFFFFFFFFF24
:101CD0007FFFFFFFFFFE7FFFFFFFFFFE3FFFFFFFD6
:101CE000FFFC0FFFFFFFFFF00FFFFFFFFFF03FFFC5
:101CF000FFFFFFFC7FFFFFFFFFFE600000001FFEF5
:101D0000E00000001FFFE00000001FFFE3FFFFFFF7
:101D10001FFFE3FFFFFF1FFFE3FFFFFF10FFE3FFD6
:101D2000FFFF10FFE3FFFFFF10FFE3FFFFFF18FFC0
:101D3000E3FFFFFF18FFE3FFFFFF1887E3FFFFFF4D
:101D40001887E3FFFFFF1887E3FFFFFF18C7E3FFD4
:101D5000FFFF18C7E3FFFFFF18C7E3FFFFFF18C728
:101D6000E3FFFFFF18C7E3FFFFFF18C7E3FFFFFF15
:101D700018C7E3FFFFFF18C7E3FFFFFF18C7E3FF24
:101D8000FFFF18C7E3FFFFFF18C7E3FFFFFF18C7F8
:101D9000E3FFFFFF18C7E3FFFFFF18C7E3FFFFFFE5
:101DA00018C7E3FFFFFF18C7E000000018C7E000F6
:101DB000000018C7E000000018C7FFFFFFFFF8C7CA
:101DC000FF1FFFFFF8C7FF00000000C7FF00000073
:101DD00000C7FF00000000C7FFFFFFFFFFC7FFF8BD
:101DE000FFFFFFC7FFF800000007FFF80000000733
:101DF0007FF8000000067FFFFFFFFFFE3FFFFFFFB1
:101E0000FFFC0FFFFFFFFFF00FFFFFFFFFF03FFFA3
:101E1000FFFFFFFC7FFFFFFFFFFE7FFFFFFFFFFED7
:101E2000FFFFFFFFFFFFF000007FFFFFF000007FDC
:101E3000FFFFF000007FFFFFF1FFFFFFFF0FF1FF4B
:101E4000FFFFFE0FF1FFFFFFFC0FF1FFFFFFF81F89
:101E5000F1FFFFFFF03FF1FFFFFFE07FF1FFFFFF2A
:101E6000C0FFF1FFFFFF81FFF1FFFFFF03FFF1FF65
:101E7000FFFE07FFF1FFFFFC0FFFF1FE1FF81FFF42
:101E8000F1FE0FF03FFFF1FE07E07FFFF1FE03C020
:101E9000FFFFF1FF0181FFFFF1FF8003FFFFF1FF73
:101EA000C007FC7FF1FFE00FFC7FF1FFF01FFC7F1C
:101EB000F1FFF83FFC7FF1FFFC7FFC7FF1FFFFFFAC
:101EC000FC7FF1FFFFFFFC7FF1FFFFFFFC7FF1FFD5
:101ED000FFFFFC7FF1FFFFFFFC7FF1FFFFFFFC7FB7
:101EE000F1FFFFFFFC7FF1FFFFFFFC7FF1FFFFFF32
:101EF000FC7FF0000000007FF0000000007FF00099
:101F00000000007FFFFFFFFFFFFFFFFFFFFFFFFF5E
:101F10007FFFFFFFFFFE7FFFFFFFFFFE3FFFFFFF93
:101F2000FFFC0FFFFFFFFFF00FFFFFFFFFF03FFF82
:101F3000FFFFFFFC7FFFFFFFFFFE7FFFFFFFFFFEB6
:101F4000FFFFFFFFFFFFFFFFFF1FFFFFFFFFFE0F72
:101F5000FFFFFFFFFE0FFFFFFFFFFE0FFFFFFFFF73
:101F6000FF1FFFFFFFFFFFFFFFFFFFFFFFFFFFFF61
:101F7000FFFFFFFFFFFFFFFFFFFFFFFFFFFFFFFF71
:101F8000FFFFFFFFC00FFFFFFFFF8007FFFFFFFF07
:101F90000007FFFFFFFE0F87FFFFFFFE1FC7FFFFCA
:101FA000FFFE3FC7FFFFFFFE3FC7FFFFFFFFFFC76B
:101FB000FFFFFFFFFFC7FFFFFFFFFFC7FFFFFFFFA1
:101FC000FF87FFFFFFFFFF0FFFFFFFFFFE1FFFFF6A
:101FD000FFFFFC3FFFFFFFFFF87FFFFFFFFFF0FF6A
:101FE000FFFFFFFFF1FFFFFFFFFFF1FFFFFFFFFF1D
:101FF000F1FFFFFFFFFFF1FFFFFFFFFFF1FFFFFF1B
:10200000FFFFF1FE3FFFFFFFF0FE3FFFFFFFF87C09
:102010003FFFFFFFFC003FFFFFFFFE007FFFFFFFD2
:10202000FF00FFFFFFFFFFFFFFFFFFFFFFFFFFFFBF
:102030007FFFFFFFFFFE7FFFFFFFFFFE3FFFFFFF72
:10204000FFFC0FFFFFFFFFF00FFFFFFFFFF03FFF61
:10205000FFFFFFFC7FFFC001FFFE7FFE00007FFE51
:10206000FFF800001FFFFFE0000007FFFFC0400275
:1020700003FFFF81800181FFFF078420E0FFFE0F47
:102080000C30F07FFC1E0C38783FF83E1C387C1F6B
:10209000F87C1C3C3E1FF07C3C3C3F0FF0FC3C3E7F
:1020A0001F0FE1F87C3E1F87E1F87C3E1F87E1F8B7
:1020B0007C3F1FC7C3F8FC3F0FC3C3F0FC3F0FC3F7
:1020C000C3F0FC3F0FC3C00000000003C0000000CD
:1020D0000003C00000000003C00000000003C7F0C0
:1020E000FC3F0FE3C3F0FC3F0FE3C3F0FC3F0FC323
:1020F000C3F0FC3F0FC3C3F0FC3F0FC3E1F8FC3F4C
:102100001FC7E1F87C3E1F87E1F87C3E1F87F0FC8B
:102110007C3E3F0FF07C3C3C3E0FF87C3C3C3E1F3D
:10212000FC3E1C387C3FFC1E0C30783FFE0F0C3010
:10213000F07FFF030420C0FFFF81800181FFFFC00B
:10214000000003FFFFF000000FFFFFF800001FFF7B
:102150007FFE00007FFE7FFFC003FFFE3FFFFFFF0B
:10216000FFFC0FFFFFFFFFF00FFFFFFFFFF03FFF40
:10217000FFFFFFFC7FFFFFFFFFFE7FFFF00FFFFE73
:10218000FFFFF00FFFFFFFFFE007FFFFFFFFC3C3ED
:10219000FFFFFFFF87E1FFFFFFFF0FF0FFFFFFFEE5
:1021A0001FF87FFFFFFC3FFC3FFFFFF87FFE1FFF94
:1021B000FFF0FFFF0FFFFFE1FFFF87FFFFE3FFFFE0
:1021C000C7FFFFE3FFFFC7FFFFE3FFFFC7FFFFE31B
:1021D000FFFFC7FFFFE3FFFFC7FFFFE3FFFFC7FFEF
:1021E000FFE3FFFFC7FFFFE3FFFFC7FFFFE3FFFFC3
:1021F000C7FFFFE3FFFFC7FFFFE3FFFFC7FFFFE3EB
:10220000FFFFC7FFFFE3FFFFC7FFFFE3FFFFC7FFBE
:10221000FFE3FFFFC7FFFFE3FFFFC7FFFFE3FFFF92
:10222000C7FFFF83FFFFC1FFFF07FFFFE0FFFE1FA8
:10223000FFFFF87FFC3FFFFFFC3FFC000000003F7A
:10224000FC000000003FFC000000003FFFFFFFFF1C
:10225000FFFFFFFFC003FFFFFFFFC003FFFFFFFF04
:10226000E007FFFFFFFFE007FFFFFFFFF81FFFFF93
:102270007FFFF81FFFFE7FFFFFFFFFFE3FFFFFFF17
:10228000FFFC0FFFFFFFFFF00FFFFFFFFFF03FFF1F
:10229000FFFFFFFC7FFFFFFFFFFE7FFFFFFFFFFE53
:1022A000F0000000000FF0000000000FF000000040
:1022B000000FF1FFFFFFFF8FF1FFFFF8888FF1FFA5
:1022C000FFF8888FF1FFFFF8888FF1FFFFFFFF8F86
:1022D000F0000000000FF0000000000FF000000010
:1022E000000FF1FFFFFFFF8FF1FFFFFFFF8FF18F67
:1022F000FFFFFF8FF187FFFFFF8FF1E3FFFFFF8FEE
:10230000F1F1FFFFFF8FF1F0FFFFFF8FF1F1FFFF12
:10231000FF8FF1E3FFFFFF8FF187FFFFFF8FF18F4B
:10232000FFFFFF8FF1FFC0FFFF8FF1FFC0FFFF8FA7
:10233000F1FFC0FFFF8FF1FFFFFFFF8FF1FFFFFFF6
:10234000FF8FF1FFFFFFFF8FF1FFFFFFFF8FF1FF17
:10235000FFFFFF8FF1FFFFFFFF8FF1FFFFFFFF8FF9
:10236000F1FFFFFFFF8FF1FFFFFFFF8FF1FFFFFF87
:10237000FF8FF1FFFFFFFF8FF1FFFFFFFF8FF000E7
:102380000000000FF0000000000FF0000000000F40
:102390007FFFFFFFFFFE7FFFFFFFFFFE3FFFFFFF0F
:1023A000FFFC0FFFFFFFFFF00FFFFFFFFFF03FFFFE
:1023B000FFFFFFFC7FFFFF803FFE7FFFFF003FFE30
:1023C000FFFFFE007FFFFFFFFC00FFFFFFFFF801A4
:1023D000FFFFFFFFF003FFFFFFFFE007FFFFFFFF2F
:1023E000C007FFFFFFFFC007FFFFFFFFC007FFFFA2
:1023F000FFFFC007FFFFFFFFC007FFFFFFFFC00792
:10240000FFE7FFFFC007FFC7FFFFC007FF87FFFF12
:10241000C007FF07FFFFC007FE07FFFFC000000760
:10242000FFFFC0000007FFFFC000000FFFFF80009C
:10243000000FFFFF0000001FFFFE0000003FFFFC39
:102440000000007FFFF8000000FFFFF0000001FF28
:10245000FFE0000003FFFFC0000007FFFF80007FD8
:10246000FFFFFF0000FFFFFFFE0001FFFFFFFC007A
:1024700003FFFFFFF80007FFFFFFF0000FFFFFFF64
:10248000E0001FFFFFFFC3803FFFFFFF87C07FFF0C
:10249000FFFF87C0FFFFFFFF87C1FFFFFFFF8383B1
:1024A000FFFFFFFFC007FFFFFFFFC00FFFFFFFFFA2
:1024B000601FFFFFFFFE783FFFFFFFFE3FFFFFFFB4
:1024C000FFFC0FFFFFFFFFF00FFFFFFFFFF03FFFDD
:1024D000FFFFFFFC7FFFFFFFFFFE7FC7FFFFF1FE57
:1024E000FF03FFFFE07FFE03FFFFE03FFC03FFFF72
:1024F000E01FF807F007F00FF00F8000F807E01E6C
:1025000000003C03E03C00001E03E07000000703F5
:10251000E0E000000383F1C001C001C7FF8003E0D9
:1025200000FFFF8003E000FFFF0003E0007FFF00EB
:1025300003E0007FFE0003E0003FFE0003E0003FF9
:10254000FC0003E0001FFC0003E0001FFC0003E0B0
:10255000001FFC0003E0001FFC0003E0001FFC0064
:1025600003F0001FFC0001F8001FFC0000FC001F2E
:10257000FC00003E001FFE00001F003FFE00000F99
:10258000803FFF000007803FFF000003007FFF80C7
:10259000000000FFFF80000000FFFF80000000FF40
:1025A000FF000000007FFE000000003FFC00000074
:1025B000001FFC060000301FFC0F8000F81FFE1FEC
:1025C000F007FC3FFFFFFFFFFFFFFFFFFFFFFFFFE5
:1025D0007FFFFFFFFFFE7FFFFFFFFFFE3FFFFFFFCD
:1025E000FFFC0FFFFFFFFFF00FFFFFFFFFF03FFFBC
:1025F000FFFFFFFC7FFFF83FFFFE7FFFF01FFFFEA6
:10260000FFFFE38FFFFFFFFFE7CFFFFFFFFFE7CFF6
:10261000FFFFFFFFE7CFFFFFFFFFE1CFFFFFFFFF60
:10262000E1CFFFFFFFFFE7CFFFFFFFFFE7CFFFFF98
:10263000FFFFE7CFFFFFFFFFE7CFFFFFFFFFE1CF88
:10264000FFFFFFFFE1CFFFFFFFFFE7CFFFFFFFFF30
:10265000E7CFFFFFFFFFE7CFFFFFFFFFE7CFFFFF62
:10266000FFFFE1CFFFFFFFFFE1CFFFFFFFFFE7CF5E
:10267000FFFFFFFFE7CFFFFFFFFFE3CFFFFFFFFFFE
:10268000E0CFFFFFFFFFE00FFFFFFFFFE00FFFFFC7
:10269000FFFFE00FFFFFFFFFE00FFFFFFFFFE00F77
:1026A000FFFFFFFFE00FFFFFFFFFE00FFFFFFFFF58
:1026B000E00FFFFFFFFFC007FFFFFFFF8003FFFFEB
:1026C000FFFF8003FFFFFFFF8003FFFFFFFF80038B
:1026D000FFFFFFFF8003FFFFFFFF8003FFFFFFFF00
:1026E000C007FFFFFFFFC007FFFFFFFFE00FFFFF77
:1026F0007FFFF01FFFFE7FFFFFFFFFFE3FFFFFFF9B
:10270000FFFC0FFFFFFFFFF00FFFFFFFFFF03FFF9A
:10271000FFFFFFFC7FFFFFFFFFFE70003FFFFFFE9C
:10272000F0001FFFFFFFF0000FFFFFFFF00007FFAB
:10273000FFFFF00003FFFFFFF00001FFFFFFF00FBE
:1027400080FFFFFFF01FC07FFFFFF03FE03FFFFF74
:10275000F07FF01FFFFFF07FF00FFFFFF07FF0072B
:10276000FFFFF07FF003FFFFF03FE001FFFFF03FCE
:10277000E000FFFFF01FC0007FFFF00F80003FFF71
:10278000F80000001FFFFC0000000FFFFE0000002B
:1027900007FFFF00000003FFFF80000001FFFFC0F4
:1027A000000000FFFFE00000007FFFF00000003F9E
:1027B000FFF80000001FFFFC0000000FFFFE0000FC
:1027C0000007FFFF00000003FFFF80000007FFFF7E
:1027D000C000000FFFFFE000001FFFFFF000003F00
:1027E000FFFFF800007FFFFFFC0000FFFFFFFE007F
:1027F00001FFFFFFFF0003FFFFFFFF8007FFFFFF59
:10280000FFC00FFFFFFFFFE01FFFFFFFFFF03FFFD5
:102810007FFFFFF87FFE7FFFFFFCFFFE3FFFFFFF14
:10282000FFFC0FFFFFFFFFF0000007E01FF8181884
:102830001818181800003FFC3C3C3C3C3C3C3E7CDB
:102840003E7C3FFC3FFC00000400060007000F0038
:102850000F801F803F907F187F1C7E3C7C3E787EDF
:1028600078FE31FE11FC09F80FE01FF83FFC7FFEF7
:10287000FFE6FFCEFF9FF33FF07FF8FFFDFE7FFEF8
:102880007FFC3FF81FF003C000E003C00F001C38BE
:1028900010F003C00F001C3810F003E007E007E061
:1028A0000000000003C003800180018001801990B6
:1028B00039B8318C618C618660066006600E700CE0
:1028C000301C1C780FF003C00380038003C007C0D6
:1028D00007E00FE00E701E701E701E783FF83FFC80
:1028E0007E7C7E7E7FFE7FFE1140820021208FE075
:1028F00023FC82004A23E200FE209FF013F8808030
:102900002220C0804221BFF0FBFA88800220848010
:10291000022084801A208080E3FE82800201010070
:102920000F421FC0784110400840904008421FC02D
:1029300008411040FFFD104008405FC00840800083
:1029400008413FE008432520104125201041252063
:102950002041252040417FF07FF848800200490057
:102960000201FFF00201001002027F20220041005C
:1029700023F07F00220008002200FF8022008880D0
:102980002200888022008A8022008900FFFC080043
:1029900023F21FC022111040FBF0904022121FC0F2
:1029A0002A11104033F1104060005FC0AFFC80007E
:1029B00020413FE022432520227925202241252065
:1029C000A541252048FD7FF01083DFC010825040D4
:1029D000208250402FFFDFC06082520061C252004F
:1029E000A1C25FE022A3D20022A251002492510092
:1029F000288E5090308BD450208258302080101078
:102A0000104047C017FC44402003F44023F84440E2
:102A10006208C440A3F8E440200154402FFD444024
:102A20002806444023F84440204044502040485069
:102A3000214050302080400020921FC03DF990403E
:102A40002090904040901FC07BFF0000A0013FE01D
:102A500021F90200FD09020021097FF021F905009A
:102A6000210945002909888031F9107021082020AA
:102A70003E0053656C65637420546970000000006B
:102A800000003E5B4F5B3E3E6B4F6B3E1C3E7C3E10
:102A90001C183C7E3C181C577D571C1C5E7F5E1C1E
:102AA00000183C1800FFE7C3E7FF0018241800FFD8
:102AB000E7DBE7FF30483A060E2629792926407FD2
:102AC000050507407F05253F5A3CE73C5A7F3E1CE1
:102AD0001C08081C1C3E7F14227F22145F5F005FCD
:102AE0005F06097F017F006689956A6060606060AB
:102AF00094A2FFA29408047E040810207E201008EF
:102B0000082A1C08081C2A08081E101010100C1E89
:102B10000C1E0C30383E3830060E3E0E060000000B
:102B2000000000005F00000007000700147F147F12
:102B300014242A7F2A12231308646236495620502F
:102B40000008070300001C2241000041221C002A4B
:102B50001C7F1C2A08083E08080080703000080806
:102B6000080808000060600020100804023E514977
:102B7000453E00427F400072494949462141494D46
:102B8000331814127F1027454545393C4A494931CD
:102B900041211109073649494936464949291E004C
:102BA00000140000004034000000081422411414F6
:102BB000141414004122140802015909063E415D13
:102BC000594E7C1211127C7F494949363E414141A0
:102BD000227F4141413E7F494949417F090909011D
:102BE0003E414151737F0808087F00417F4100202A
:102BF00040413F017F081422417F404040407F0216
:102C00001C027F7F0408107F3E4141413E7F09093D
:102C100009063E4151215E7F091929462649494945
:102C20003203017F01033F4040403F1F2040201FEF
:102C30003F4038403F631408146303047804036181
:102C400059494D43007F4141410204081020004191
:102C500041417F040201020440404040400003071C
:102C6000080020545478407F284444383844444471
:102C700028384444287F385454541800087E0902E8
:102C800018A4A49C787F0804047800447D400020A8
:102C900040403D007F1028440000417F40007C04FC
:102CA0007804787C080404783844444438FC1824B8
:102CB000241818242418FC7C08040408485454548C
:102CC0002404043F44243C4040207C1C2040201C21
:102CD0003C4030403C44281028444C9090907C4428
:102CE00064544C4400083641000000770000004165
:102CF00036080002010204023C2623263C1EA1A144
:102D000061123A4040207A3854545559215555792A
:102D100041215454784121555478402054557940EC
:102D20000C1E52721239555555593954545459394B
:102D3000555454580000457C410002457D42000135
:102D4000457C40F0292429F0F0282528F07C5455B2
:102D500045002054547C547C0A097F493249494932
:102D6000323248484832324A4848303A4141217A62
:102D70003A42402078009DA0A07D39444444393D2A
:102D80004040403D3C24FF2424487E4943662B2F8D
:102D9000FC2F2BFF0929F620C0887E0903205454FC
:102DA00079410000447D413048484A323840402251
:102DB0007A007A0A0A727D0D19317D2629292F2879
:102DC000262929292630484D4020380808080808B7
:102DD000080808382F10C8ACBA2F102834FA0000A1
:102DE0007B000008142A142222142A1408950022B9
:102DF0000095AA005500AAAA55AA55AA000000FFEE
:102E000000101010FF00141414FF001010FF00FF3A
:102E10001010F010F0141414FC001414F700FF004C
:102E200000FF00FF1414F404FC141417101F1010FA
:102E30001F101F1414141F00101010F000000000C9
:102E40001F101010101F10101010F010000000FFC5
:102E5000101010101010101010FF10000000FF14C0
:102E60000000FF00FF00001F10170000FC04F41416
:102E7000141710171414F404F40000FF00F71414CE
:102E80001414141414F700F7141414171410101F4A
:102E9000101F141414F4141010F010F000001F1080
:102EA0001F0000001F14000000FC140000F010F0D0
:102EB0001010FF10FF141414FF141010101F000046
:102EC0000000F010FFFFFFFFFFF0F0F0F0F0FFFF59
:102ED000FF0000000000FFFF0F0F0F0F0F384444EA
:102EE00038447C2A2A3E147E02020606027E027EB6
:102EF0000263554941633844443C04407E201E200F
:102F000006027E020299A5E7A5991C2A492A1C4CB3
:102F10007201724C304A4D4D303048784830BC62B6
:102F20005A463D3E494949007E0101017E2A2A2A2E
:102F30002A2A44445F444440514A444040444A5150
:102F4000400000FF0103E080FF000008086B6B08F1
:102F50003612362436060F090F0600001818000036
:102F6000001010003040FF0101001F01011E001978
:102F70001D1712003C3C3C3C00000000000000001B
:102F800000240027002A0000000000250028002B54
:102F900000000000002300260029000404040404AB
:102FA00004040402020202020203030303030301F6
:102FB00002040810204080010204081020010204CD
:102FC000081020AED5F0A83FD300408D14A1C8DA78
:102FD0001281CFD9F1DB40A4A6AF200021007F22CF
:102FE0000007506C65617365207761697400414426
:102FF000433A200074656D703A2000536574206D6B
:103000006561737572656400537465703A200000E1
:10301000003E0E7C0C000000003E0E7C0C00000008
:10302000003E0E7C0C00001FFE3FC18C0C7FF81F81
:10303000FE3FC18C0C7FF818063001F38C60181825
:10304000063001F38C601818063001F38C601818F4
:10305000063E0FF00C601818063E0FF00C601818B2
:10306000063FC1F00C601818063FC1F00C6018183C
:10307000063FC1F00C60181FFE3E30700C7FF81F39
:10308000FE3E30700C7FF8000031CE738C000000E3
:103090000031CE738C0000000031CE738C0000FF35
:1030A000FFF001838FFFFFFFFFF001838FFFFF0021
:1030B000C001C18C007F1F00C001C18C007F1F00B8
:1030C000C001C18C007F1F07C7CFCE7F8C1FF807C0
:1030D000C7CFCE7F8C1FF807C7CFCE7F8C1FF8F8E5
:1030E000003E3E03F07F00F8003E3E03F07F00E02C
:1030F000C7CFFE03801FE7E0C7CFFE03801FE7E0D6
:10310000C7CFFE03801FE718C031FE0C0C1CE0186F
:10311000C031FE0C0C1CE0E739F1F003FC7CF8E751
:1031200039F1F003FC7CF8E739F1F003FC7CF81F7F
:103130000031CFF38C03001F0031CFF38C0300E08C
:103140003FFFC1838F9CE7E03FFFC1838F9CE7E097
:103150003FFFC1838F9CE71800300E000000FF186E
:1031600000300E000000FF1800300E000000FFFFCE
:10317000FFF03E7C0FE000FFFFF03E7C0FE0000020
:103180000031CE0C0C63E0000031CE0C0C63E0008B
:103190000031CE0C0C63E01FFE3001838FE0FF1F77
:1031A000FE3001838FE0FF180631F18F8003E718AE
:1031B0000631F18F8003E7180631F18F8003E7189D
:1031C000063FFF8383E31F18063FFF8383E31F1837
:1031D0000631FE738F80F8180631FE738F80F81861
:1031E0000631FE738F80F81FFE31FE000C60E71F72
:1031F000FE31FE000C60E7000031FE0C0F9FE00086
:103200000031FE0C0F9FE0000031FE0C0F9FE02507
:10321000004300202070F83030300076312E364CDC
:10322000310056005600430000800080018001807C
:103230000380078007F00FF00FE01FC001C001807E
:103240000180018001000100124812481FF8E007C8
:103250002E142C04E80720042004E007200428147E
:10326000E0071FF8124812484552524F5200484F8B
:103270004C44004845415400574F524B5900424F6F
:103280004F535400534C454550004F4646000000F4
:103290007E007F00738061C061E073F03FF81FFC27
:1032A0000FFE07FF03FF01FE00FC00780030303006
:1032B00030000102040810204080000000080002D5
:1032C00001000003040700000000000000001A2DA8
:1032D00011241FBECFEFD8E0DEBFCDBF12E0A0E0CB
:1032E000B1E0EEEBFAE702C005900D92A237B1070C
:1032F000D9F727E0A2E7B2E001C01D92AD3AB207CC
:10330000E1F719E1C8E6D9E104C02197FE010E9466
:10331000603BC736D107C9F70E94CF2D0C945D3DA5
:103320000C9400004F925F926F927F928F929F92C7
:10333000AF92BF92CF92DF92EF92FF920F931F93C3
:10334000CF93DF9300D000D0CDB7DEB74B015C0147
:1033500029013A016701780120E030E0A9010E94CB
:10336000653887FDA6C020E030E0A901C301B201A5
:103370000E94653887FD9DC020E030E0A901C801AA
:10338000B6010E94653887FD94C081E020917307E3
:10339000309174072130310509F080E08093940763
:1033A0008092590790925A07A0925B07B0925C07EF
:1033B00040925D0750925E0760925F0770926007CF
:1033C000C0926107D0926207E0926307F0926407AF
:1033D00060918707709188078091890790918A078B
:1033E0000E946A3820E030E04AE754E40E949E3AA6
:1033F00069837A838B839C838092650790926607AA
:10340000A0926707B09268079B01AC01C301B201AB
:103410000E94CB382B013C014092690750926A0709
:1034200060926B0770926C0729813A814B815C81B5
:10343000C701B6010E949E3A6B017C01C0926D07E4
:10344000D0926E07E0926F07F0927007809171073B
:1034500090917207019769F5A501940160E070E011
:10346000CB010E94313A60936507709366078093A1
:10347000670790936807A301920160E070E0CB01B9
:103480000E94313A6093690770936A0780936B07D3
:1034900090936C07A701960160E070E0CB010E9459
:1034A000313A60936D0770936E0780936F07909326
:1034B00070070F900F900F900F90DF91CF911F9199
:1034C0000F91FF90EF90DF90CF90BF90AF909F90C3
:1034D0008F907F906F905F904F9008958038910506
:1034E000B0F46034710598F4E2EBF2E390E1969F5A
:1034F000D001A0781124A80F6770E60FF11D9491F8
:10350000A055BD4F442321F08C91982B9C93089596
:1035100090958C919823FACF2F923F924F925F9281
:103520006F927F928F929F92AF92BF92CF92DF92D3
:10353000EF92FF920F931F93CF93DF9300D01F92D0
:10354000CDB7DEB7C22ED12C9601280F391F37FD1B
:103550004FC0803891050CF04BC0E9824A017B01D5
:103560003C01402E512C160127E0220E311C93E025
:10357000359427949A95E1F78B01B12CA12C1B82ED
:103580001A82EA81FB8183E0F595E7958A95E1F758
:10359000EA0DFB1DE80DF91DE4918A819B8187707E
:1035A000992720E830E002C0359527958A95E2F703
:1035B000C901F0E0E223F923EF2B41F04981B80182
:1035C0008A819B81860D971D0E946E1A8A819B813C
:1035D00001969B838A838C159D059CF2A20CB31CDB
:1035E0000F5F1F4FC8018E199F09841595053CF286
:1035F0000F900F900F90DF91CF911F910F91FF903F
:10360000EF90DF90CF90BF90AF909F908F907F9082
:103610006F905F904F903F902F90089580E0E0EB87
:10362000F2E081118FEF0024819381938193819344
:103630000394D1F7E5E9F7E0178616861586148618
:103640000895DF92EF92FF920F931F93CF93DF9332
:103650007C01EB01D22E8B01040F111DC801013436
:10366000110514F080E490E0C817D9073CF44D2D03
:10367000BE01C7010E946E1A2196F0CFDF91CF9153
:103680001F910F91FF90EF90DF900895CF92DF92FE
:10369000EF92FF920F931F93CF93DF936B01122F43
:1036A000EC017C01E40EF11CCE15DF0544F4202F63
:1036B000412FB601CE010E94211B2196F5CFDF914B
:1036C000CF911F910F91FF90EF90DF90CF900895D1
:1036D000480F592F511D4138510514F040E850E072
:1036E000481BFB01E770FF2721E030E001C0220FFB
:1036F000EA95EAF7209577FF02C0695F7F4FFB01EB
:1037000033E0F595E7953A95E1F7F695FE2FEE272C
:10371000F795E795E80FF91FE055FD4F415030F060
:103720008191DF01119782238C93F8CF0895EF9256
:10373000FF920F931F93CF93DF937C018B01C42FD4
:10374000D22F0E94681BB8016D0F711D6150710965
:103750006034710524F44C2FC7010E94681B20E0DF
:103760004D2FB801C7010E94211BC7018C0F911D6D
:1037700020E04D2FB8010197DF91CF911F910F915C
:10378000FF90EF900C94211B0895AF92BF92CF92BF
:10379000DF92EF92FF920F931F93CF93DF936C0111
:1037A0007B018B01040F151FEB015E01AE18BF08F2
:1037B000C017D10759F06991D601ED91FC910190A4
:1037C000F081E02DC6010995892B79F7C501DF91BC
:1037D000CF911F910F91FF90EF90DF90CF90BF900E
:1037E000AF900895FC01538D448D252F30E0842F38
:1037F00090E0821B930B541710F0CF960895019719
:103800000895FC01918D828D981761F0A28DAE0F05
:10381000BF2FB11D5D968C91928D9F5F9F73928F8C
:1038200090E008958FEF9FEF0895FC01918D828DB8
:10383000981731F0828DE80FF11D858D90E0089585
:103840008FEF9FEF0895FC01918D228D892F90E0DD
:10385000805C9F4F821B91098F739927089580EB9D
:1038600096E00E94231C21E0892B09F420E0822F9E
:10387000089580E090E0892B29F00E942F1C81118F
:103880000C9400000895FC01A48DA80FB92FB11D60
:10389000A35ABF4F2C91848D90E001968F73992786
:1038A000848FA689B7892C93A089B1898C91837064
:1038B00080648C93938D848D981306C00288F3895D
:1038C000E02D80818F7D80830895EF92FF920F938A
:1038D0001F93CF93DF93EC0181E0888F9B8D8C8DBC
:1038E00098131AC0E889F989808185FF15C09FB7B0
:1038F000F894EE89FF896083E889F9898081837073
:10390000806480839FBF81E090E0DF91CF911F9121
:103910000F91FF90EF900895F62E0B8D10E00F5F42
:103920001F4F0F731127E02E8C8D8E110CC00FB618
:1039300007FCFACFE889F989808185FFF5CFCE01B0
:103940000E94431CF1CFEB8DEC0FFD2FF11DE35ACC
:10395000FF4FF0829FB7F8940B8FEA89FB89808133
:103960008062CFCFCF93DF93EC01888D8823B9F0AD
:10397000AA89BB89E889F9898C9185FD03C080817A
:1039800086FD0DC00FB607FCF7CF8C9185FFF2CFF7
:10399000808185FFEDCFCE010E94431CE9CFDF91EE
:1039A000CF910895833081F028F4813099F08230EE
:1039B000A9F008958730A9F08830C9F08430B1F4B7
:1039C000809180008F7D03C0809180008F778093ED
:1039D0008000089584B58F7784BD089584B58F7D68
:1039E000FBCF8091B0008F778093B00008958091D5
:1039F000B0008F7DF9CFCF93DF93282F30E0F9010E
:103A0000E654FD4C8491F901E155F04DD491F90152
:103A1000E556F04DC491CC23A1F081110E94D21C37
:103A2000EC2FF0E0EE0FFF1FEF56F04DA591B49193
:103A3000EC91ED2381E090E009F480E0DF91CF91FB
:103A4000089580E090E0FACF1F93CF93DF93282F63
:103A500030E0F901E654FD4C8491F901E155F04D57
:103A6000D491F901E556F04DC491CC23A9F0162F5D
:103A700081110E94D21CEC2FF0E0EE0FFF1FE957DE
:103A8000F04DA591B4918FB7F894EC91111108C045
:103A9000D095DE23DC938FBFDF91CF911F910895E6
:103AA000DE2BF8CFCF93DF9390E0FC01E155F04D92
:103AB00024918556904DFC0184918823C9F090E0B3
:103AC000880F991FFC01E358F04DA591B491FC01BA
:103AD000E957F04DC591D49161110DC09FB7F8948D
:103AE0008C91209582238C938881282328839FBFE3
:103AF000DF91CF910895623051F49FB7F8943C91D3
:103B0000822F809583238C93E8812E2BEFCF8FB764
:103B1000F894EC912E2B2C938FBFEACFCF93DF93A9
:103B2000EC0161E089E00E94521D209731F460E0D1
:103B300089E0DF91CF910C94241DCF3FD10511F482
:103B400061E0F6CFE3ECF2E3E491E33029F140F4F5
:103B5000E130B1F0E230D9F0C038D1058CF7E7CFD1
:103B6000E73021F1E83051F1E430B1F78091800085
:103B7000806280938000D0938B00C0938A0004C041
:103B800084B5806884BDC7BDDF91CF91089584B5A9
:103B9000806284BDC8BDF8CF80918000806880932A
:103BA0008000D0938900C0938800EECF8091B00050
:103BB00080688093B000C093B300E6CF8091B000DE
:103BC00080628093B000C093B400DECF3FB7F8941A
:103BD0008091790290917A02A0917B02B0917C024F
:103BE00026B5A89B05C02F3F19F00196A11DB11D58
:103BF0003FBFBA2FA92F982F8827BC01CD01620F94
:103C0000711D811D911D42E0660F771F881F991F4E
:103C10004A95D1F708958F929F92AF92BF92CF921B
:103C2000DF92EF92FF924B015C010E94E61D6B0157
:103C30007C010E94E61D6C197D098E099F09683E72
:103C4000734081059105A8F321E0821A9108A1082B
:103C5000B10888EEC80E83E0D81EE11CF11C811467
:103C60009104A104B10429F7FF90EF90DF90CF9069
:103C7000BF90AF909F908F9008952FB7F894609168
:103C800075027091760280917702909178022FBF31
:103C9000089584E98093BC008091BC0084FDFCCF32
:103CA00008958093BB0084E88093BC008091BC00A1
:103CB00087FFFCCF089584EA8093BC008091BC000C
:103CC00087FFFCCF88E70C94511E0E945B1E80E4A6
:103CD0008093BB0084E88093BC00E0EBF2E090911D
:103CE000BC0097FFFCCF91919093BB008093BC00E8
:103CF00096E0E03BF90799F78091BC0087FFFCCF85
:103D00000C94491ECF93C82F0E945B1E80E00E9436
:103D1000511E8C2F0E94511ECF910C94491E2F9240
:103D20003F924F925F926F927F928F929F92AF924B
:103D3000BF92CF92DF92EF92FF920F931F93CF9398
:103D4000DF93CDB7DEB72A970FB6F894DEBF0FBE6C
:103D5000CDBF9A8389836A3061F5DC0152968C91DC
:103D6000B8E08B9F90011124E981FA8186859785BF
:103D7000820F931F978786871586148681E090E0CF
:103D80002A960FB6F894DEBF0FBECDBFDF91CF915C
:103D90001F910F91FF90EF90DF90CF90BF90AF9069
:103DA0009F908F907F906F905F904F903F902F905B
:103DB00008956D3019F329813A813A872987D9010D
:103DC0001C96AD90BC90B0E8AB16B1040CF07BC073
:103DD000F901C684D784F0E4CF16D1040CF073C087
:103DE000D90152966C90529745E09501649E200D42
:103DF000311D1124121613060CF065C0262C312C2F
:103E0000910153E0220F331F5A95E1F72C0D3D1D10
:103E1000121613060CF057C05196BC91BB83E9856E
:103E2000FA85F089FC83649FB00111249B0123581B
:103E3000354D3A832983712CE981FA818491F5E02B
:103E40007F1201C080E0460138E0532E282F30E079
:103E50003E832D834C8080FF4B80411004C03B810A
:103E60008C813817E1F010E000E00615C0F4D501B0
:103E7000A00FB11FB887AF83F12CE12CE61460F4DA
:103E8000B701680D791D442D8F8198850E946E1AA7
:103E9000BFEFEB1AFB0AF2CF0F5F1F4FE6CF8D810A
:103EA0009E81959587955A94820C931C5110CECF84
:103EB0007394E981FA813196FA83E983A20CB31CE9
:103EC000F6E07F12B9CFA985BA8552962C91529708
:103ED000422F50E01C968D919C91B6E02B9F800D57
:103EE000911D1124E985FA859587848723892223EA
:103EF00009F444CF6AEF64039001659F300D1124EB
:103F000020583F4F281739070CF038CFDF010190B8
:103F1000F081E02D0190F081E02D6AE0CD0109955E
:103F20002DCF682F85E997E00C948F1E0F931F9378
:103F3000CF93DF938C01D0E0C0E0F801EC0FFD1FC0
:103F40006491662341F085E997E00E948F1E892BDA
:103F500011F02196F2CFCE01DF91CF911F910F91F9
:103F6000089590E080E0089580917A0080698093C0
:103F70007A008EE480937C0061E070E080E090E065
:103F80000E940B1E83B7817F826083BF80E130E097
:103F900020E093B7916093BF889593B79E7F93BFBE
:103FA00090917A0096FDFCCF409178005091790075
:103FB000240F351F815069F780917A008F778093A5
:103FC0007A0084E0369527958A95E1F750E040E045
:103FD00064EB7BE281E190E00E949F39C901089582
:103FE00080917A00806980937A0088EC80937C00CD
:103FF00064E170E080E090E00E940B1E83B7817F57
:10400000826083BF80E270E060E093B7916093BF0D
:10401000889593B79E7F93BF90917A0096FDFCCFD1
:104020002091780030917900620F731F815069F7F9
:1040300080917A008F7780937A0076956795769550
:10404000679562527A4090E080E00E946A3826EFDD
:1040500038E24CE151E40E949E3A089590917A0032
:10406000906990937A008E50806480937C0083B72F
:10407000817F826083BF20E290E080E033B73160CF
:1040800033BF889533B73E7F33BF30917A0036FD1A
:10409000FCCF4091780050917900840F951F2150FA
:1040A00069F720917A002F7720937A0025E0969582
:1040B00087952A95E1F708958FE00E942E20A09120
:1040C0008002B09181029C010E94223A0E946C38C9
:1040D00028E539E743E353E40E949E3A0E94173BE8
:1040E000CB01089580918702882369F086E00E94C1
:1040F000FB1C892B41F06AE070E080E090E00E94B8
:104100000B1E1092870208950F931F93CF938091F7
:104110004801882399F0CFEF0FEE11E061E085E0D0
:104120000E94241DC8010197F1F760E085E00E941C
:10413000241DC8010197F1F7C15081F7CF911F915C
:104140000F9108952F923F924F925F926F927F92BC
:104150008F929F92AF92BF92CF92DF92EF92FF9297
:104160000F931F93CF93DF9310E000E0D0E0C0E007
:104170003EE3E32EF12C40ECC42ED12CAA24A394D0
:10418000B12C60E2662E712C70E4272E312C4C2E5F
:1041900086E00E94FB1C21E0892B09F020E020939F
:1041A0008702F0928D02E0928C02D0928B02C09234
:1041B0008A02B0928902A092880282E890E09093ED
:1041C0009902809398028091980290919902959516
:1041D0008795582E9FE1591243C0F0928D02E092CC
:1041E0008C02D0928B02C0928A02B0928902A09275
:1041F0008802EEEBF0E0F0939902E09398029FE5DD
:10420000592E0E940E1B82E08093A7071093A207ED
:104210000093A107E0E3F0E0F093A407E093A30785
:104220008EE50E94911F1092A2071092A107709232
:10423000A4076092A307912C812C841438F58091F7
:10424000AC02F40196E0989FE00DF11D1124E15BB2
:10425000FE4F80810E94911FEFEF8E1A9E0AEDCFD4
:10426000F0E65F12CECFF0928D02E0928C02D092F7
:104270008B02C0928A02B0928902A0928802309288
:1042800099022092980280E2582EBBCF1093A20789
:104290000093A1077092A4076092A307852D0E9446
:1042A000911F0E9472200E94651E86E00E94FB1CE6
:1042B000892B09F088CF80918702811184CF80906B
:1042C000AC02F6E08F9E40011124C401815B9E4F39
:1042D0004C01FC01EC0FFD1F50820E9484206AE01B
:1042E00070E080E090E00E940B1E2196005F1F4F5F
:1042F000C530D10509F04BCFF4011582DF91CF9184
:104300001F910F91FF90EF90DF90CF90BF90AF90F3
:104310009F908F907F906F905F904F903F902F90E5
:1043200008952F923F924F925F926F927F928F9259
:104330009F92AF92BF92CF92DF92EF92FF920F9334
:104340001F93CF93DF9300D000D000D0CDB7DEB75E
:10435000B82EC0908E02D12CF601E35EFD4F408056
:1043600010928D0210928C02242D30E03A83298322
:10437000C9010197880F991F90938B0280938A023D
:1043800081E090E090938902809388028B2D90E0E9
:10439000880F991F909399028093980286E00E945B
:1043A000FB1C21E0892B09F020E02093870238E3F1
:1043B000F32E209098023090990235942794122D74
:1043C0004101992494012B193109F29EC001F39EF9
:1043D000900D11242D813E81280F391F3E832D839E
:1043E0002115310521F1B901719561957109072EEA
:1043F000000C880B990B0E946C3820E030E040E004
:104400005FE30E94CB382B013C012D813E81B90135
:10441000330F880B990B0E946C389B01AC01C301D0
:10442000B2010E94323A0E94103B7E836D830E944B
:104430000E1B540132E0A31AB1086D807E80C401C6
:1044400003969C838B8329813A81A216B30620F5BB
:10445000EDE1F2E090E080E09F012D5132402C151B
:104460003D0534F42191820F911DF6CFB22CA1CFDE
:10447000F501E80FF11DEE0FFF1FEF52FE4F4081D7
:104480005181EE24E39400E320E370E060E0C30197
:10449000885491090E948C1A3FEFA31AB30A88E34B
:1044A000680E711C2B813C81A216B30661F6EDE10A
:1044B000F2E090E080E09F012D5132402C153D0547
:1044C00024F42191820F911DF6CFF401E80FF11D24
:1044D000EE0FFF1FEB57FE4F40815181EE24E39416
:1044E00000E124E260E370E080E390E00E948C1A37
:1044F0000E94651E0E94722086E00E94FB1C892B90
:1045000009F0B4CF809187028111B0CF0E9484203E
:10451000812F26960FB6F894DEBF0FBECDBFDF9178
:10452000CF911F910F91FF90EF90DF90CF90BF90B0
:10453000AF909F908F907F906F905F904F903F9043
:104540002F9008953F924F925F926F927F928F9239
:104550009F92AF92BF92CF92DF92EF92FF920F9312
:104560001F93CF93DF93CDB7DEB72E970FB6F89496
:10457000DEBF0FBECDBF8091AB02882309F4A5C179
:1045800010924D0710924E0710924F07109250074D
:1045900080904D0790904E07A0904F07B090500725
:1045A000C090A102D090A202E090A302F090A402D9
:1045B000A7019601C501B4010E94313A2B013C01CB
:1045C00020E030E0A9010E94463B18160CF0A0C183
:1045D000C301B2010E94173B80914901882309F46D
:1045E000B8C1C0925507D0925607E0925707F09293
:1045F0005807E12CF12C00EA10E420E030E040E420
:1046000050E46E31710540F0E12CF12C00E81FE31D
:1046100020E030E040E05FE360E070E080E391E4C0
:104620000E94921980919307882309F42AC10E945D
:104630003D1E6D837E838F83988780917B07909149
:104640007C07A0917D07B0917E074D815E816F81CF
:104650007885481B590B6A0B7B0B809187079091DB
:104660008807A0918907B0918A07481759076A07F8
:104670007B0708F406C1E0917507F0917607808109
:104680009181A281B38189839A83AB83BC83E091BA
:104690007907F0917A079C01AD0160817181828177
:1046A00093810E94313A4B015C0120918307309144
:1046B0008407409185075091860769817A818B81B3
:1046C0009C810E94313A6B017C01209169073091F5
:1046D0006A0740916B0750916C07C501B4010E94B5
:1046E000CB3820917F07309180074091810750910E
:1046F00082070E94323A2B013C0140927F07509280
:104700008007609281077092820730909407311081
:104710001AC0209165073091660740916707509154
:104720006807C701B6010E94CB389B01AC01C301E9
:10473000B2010E94313A60937F07709380078093A3
:1047400081079093820740907F0750908007609088
:1047500081077090820710918F07909190079E8734
:10476000A0919107AD8700919207212F392F4A2FF1
:10477000502FC301B2010E94463B18160CF0CCC06A
:10478000812F9E85AD85B02F80937F079093800702
:10479000A0938107B0938207332009F4D6C02091FB
:1047A0006507309166074091670750916807C5011A
:1047B000B4010E94CB384B015C0120916D07309110
:1047C0006E0740916F0750917007C701B6010E94B4
:1047D000CB389B01AC0160917F077091800780917D
:1047E0008107909182070E94313AA50194010E94AD
:1047F000323A6B017C019B01AC01612F7E858D8576
:10480000902F0E94653887FD18C010918B079091FA
:104810008C079E87A0918D07AD8700918E07212F71
:10482000392F4A2F502FB601C7010E94653887FDE6
:1048300004C01C2DDE86ED860F2DE0917707F091E8
:104840007807812F9E85AD85B02F80839183A283C9
:10485000B38389819A81AB81BC81809383079093D4
:104860008407A0938507B09386078D819E81AF81D1
:10487000B88580937B0790937C07A0937D07B093C6
:104880007E07609151077091520780915307909174
:1048900054070E94103BCB012E960FB6F894DEBF52
:1048A0000FBECDBFDF91CF911F910F91FF90EF9081
:1048B000DF90CF90BF90AF909F908F907F906F9040
:1048C0005F904F903F900C948E1D8091AA02609152
:1048D00044017091450181110EC080919F02909119
:1048E000A0022091A902BC01222329F0609143017A
:1048F000680F792F711D90E080E00E946A38609304
:104900004D0770934E0780934F079093500740CE0A
:10491000C301B20190585ECE80918B0790918C07B5
:10492000A0918D07B0918E0789879A87AB87BC8746
:104930009C01AD01C301B2010E94653887FF2CCFF5
:1049400089859A85AB85BC851FCF812C912C54011C
:1049500034CF20E030E040E05FE3C701B6010E94C1
:10496000323A9B01AC01C501B4010E94463B1816C6
:104970004CF4109251071092520710925307109264
:1049800054077FCF80E090E0AFE7B3E48093510716
:1049900090935207A0935307B093540772CF4F924E
:1049A0005F926F927F928F929F92AF92BF92CF92BF
:1049B000DF92EF92FF92CF93DF93809082029090EC
:1049C0008302A0908402B0908502C091AC02D0E036
:1049D000C501B4010E94103B6B017C0120E030E076
:1049E00048E453E4C501B4010E94653893E0CC0F5C
:1049F000DD1F9A95E1F7CE5FDE4F87FF31C028813A
:104A0000398150E040E02551310941095109C70180
:104A1000B6010E94503B28EC30E040E050E00E949C
:104A20009F39CA01B9016B5E7F4F8F4F9F4F0E9424
:104A30006C386093A1027093A2028093A3029093BA
:104A4000A402DF91CF91FF90EF90DF90CF90BF90C5
:104A5000AF909F908F907F906F905F904F90089550
:104A60004A805B80712C612C20E030E04CE853E4FC
:104A7000C501B4010E94653887FF1FC088809980F6
:104A8000B12CA12CA7019601285C310941095109DB
:104A9000C301B201681979098A099B090E94503B38
:104AA00020E530E040E050E00E949F39CA01B901A2
:104AB000680D791D8A1D9B1DBACF2C813D8150E068
:104AC00040E02419350946095709C701B601685164
:104AD0007140810991090E94503B20E530E040E09F
:104AE00050E00E949F39CA01B901640D751D861DF1
:104AF000971D9DCFFC0101900020E9F73197AF0190
:104B0000481B590BBC0185E997E00C94C51B8F929B
:104B10009F92AF92BF920F931F93CF93DF93CDB726
:104B2000DEB7A1970FB6F894DEBF0FBECDBF19A2B6
:104B3000423008F44AE08E010F5D1F4F842E912C05
:104B4000B12CA12CA50194010E94003AE62FB901D5
:104B5000CA01EA30F4F4E05DD801EE938D01232B15
:104B6000242B252B79F790E080E0109719F0CD01E8
:104B70000E947A25A1960FB6F894DEBF0FBECDBF76
:104B8000DF91CF911F910F91BF90AF909F908F9029
:104B90000895E95CE1CFCF92DF92EF92FF92CF933D
:104BA000DF9397FF19C06B017C018DE20E94911F7A
:104BB000EC0166277727CB016C197D098E099F09C7
:104BC0004AE00E9487258C0F9D1FDF91CF91FF90B7
:104BD000EF90DF90CF9008954AE0DF91CF91FF9062
:104BE000EF90DF90CF900C9487254F925F926F9259
:104BF0007F928F929F92AF92BF92CF92DF92EF926D
:104C0000FF920F931F93CF936B017C01742EAC0125
:104C10009B010E944B3B882399F082E692E0CF9162
:104C20001F910F91FF90EF90DF90CF90BF90AF90CA
:104C30009F908F907F906F905F904F900C947A250B
:104C400046015701E894B7F82FEF3FEF4FE75FE7D2
:104C5000C501B4010E944B3B81110DC02FEF3FEF06
:104C60004FE75FE7C501B4010E94653818161CF4D0
:104C700086E692E0D4CF2FEF3FEF4FE75FE4C70126
:104C8000B6010E94463B18161CF48AE692E0C7CF94
:104C90002FEF3FEF4FE75FECC701B6010E94653889
:104CA00087FDF3CF20E030E0A901C701B6010E94E3
:104CB000653810E000E087FF08C08DE20E94911F78
:104CC0008C01F7FAF094F7F8F094C0E060E070E03F
:104CD00080E09FE37C1641F020E030E040E251E4C8
:104CE0000E949E3ACF5FF6CFA70196010E94323A0A
:104CF0002B013C010E94173B4B015C014AE00E94E2
:104D000087257C01E00EF11ECC23B1F1C501B40171
:104D10000E946A389B01AC01C301B2010E94313A82
:104D20004B015C018EE20E94911FE80EF91EC150FA
:104D300018F120E030E040E251E4C501B4010E94E6
:104D4000CB382B013C010E94173B4B01B12CA12C0D
:104D50004AE0C501B4010E948725E80EF91EC5018D
:104D6000B4010E946A389B01AC01C301B2010E94E8
:104D7000313A4B015C01DBCFC701CF911F910F91FD
:104D8000FF90EF90DF90CF90BF90AF909F908F906B
:104D90007F906F905F904F9008956F927F928F9267
:104DA0009F92AF92BF92CF92DF92EF92FF920F93BA
:104DB0001F93CF93DF93B090AC0277247394B1101C
:104DC00001C0712C809142018150990B10928D028B
:104DD00010928C02880F991F90938B0280938A0205
:104DE00081E090E090938902809388028B2D90E07F
:104DF000880F991F909399028093980286E00E94F1
:104E0000FB1C21E0892B09F020E020938702FF247E
:104E1000F39472E0972EE6E08E2EFCE0CF2ED12C9C
:104E20000E940E1BC0919802D0919902D595C7950A
:104E3000EC2E8E011127C801870D911D77FC9A95E4
:104E40008B199109712C97FD06C08330910514F0E0
:104E500082E090E0782EF092A6071092A50790923B
:104E6000A7071092A2071092A1071092A407109210
:104E7000A30782E79AE20E94961F1092A607F0927B
:104E8000A5071092A2071092A107A72C072C000CCF
:104E9000BB08C501019654E0880F991F5A95E1F7A8
:104EA0009093A4078093A30780E79AE20E94961F3D
:104EB0006C2E671890E080E098012A193B0959018F
:104EC000209142018C010F5F1F4F6216D0F4D092E7
:104ED000A207C092A107980144E0220F331F4A9510
:104EE000E1F73093A4072093A3078A0D9B1D889EAA
:104EF0009001899E300D1124C901815B9E4F0E9453
:104F00007A25C801639403301105D1F60E947220FE
:104F10000E94651E86E00E94FB1C892BB9F48091DB
:104F20008702811113C00E948420E092AC02DF91BD
:104F3000CF911F910F91FF90EF90DF90CF90BF9096
:104F4000AF909F908F907F906F900895BC2E68CF08
:104F50000E94483DEF92FF920F931F93CF93DF93F0
:104F6000EC017B018A0188819981009729F02A81CF
:104F70003B812417350788F4B8016F5F7F4F0E948B
:104F80008B3C009791F0998388831B830A832C8143
:104F90003D81232B11F4FC0110821D830C83B7018A
:104FA000888199810E94563D0CC088819981009723
:104FB00011F00E94023C198218821D821C821B8201
:104FC0001A82CE01DF91CF911F910F91FF90EF9048
:104FD00008951F93CF93DF93EC01162F0E94893918
:104FE000181739F0612FCE01DF91CF911F910C94EA
:104FF0009139DF91CF911F910895AF92BF92CF92D7
:10500000DF92EF92FF920F931F93CF93DF93609104
:10501000470182E090E00E94E9276091460183E029
:1050200090E00E94E9276091450184E090E00E94B1
:10503000E9276091440185E090E00E94E9276091B2
:10504000430186E090E00E94E92760914C0187E0EF
:1050500090E00E94E92760914B0188E090E00E9477
:10506000E92760914A0189E090E00E94E927609178
:10507000AF028AE090E00E94E927609149018BE04D
:1050800090E00E94E927609148018CE090E00E9446
:10509000E9276091AC028DE090E00E94E9276091E1
:1050A00042018EE090E00E94E9276091A8028FE023
:1050B00090E00E94E9276091860280E190E00E94E2
:1050C000E92781E1E82EF12C10E006E08091420111
:1050D0001817B8F5109F60011124D0E0C0E0FE0160
:1050E000EC0DFD1DE15BFE4F6081C7018C0F9D1F24
:1050F0000E94E9272196C630D10589F7670186E02D
:10510000C80ED11C88E0189FE0011124CE5FDE4F4D
:105110008EE0E80EF11C69812296C6010E94E92703
:10512000560182E0A80EB11CFE0132976081C601D3
:1051300001960E94E9276501AE14BF0461F71F5F65
:10514000C5CFDF91CF911F910F91FF90EF90DF902E
:10515000CF90BF90AF9008958F929F92AF92BF92E1
:10516000CF92DF92EF92FF92CF938FEF90E00E9469
:105170008E1D8BEA94E00197F1F78EE00E942E20BD
:105180007C018AE00E94FB1C90917202981729F022
:1051900091E09093A50280937202809101019FEFAC
:1051A000980F90930101811106C00E945C2090939A
:1051B000A7028093A60260915107709152078091D7
:1051C0005307909154070E94103BCB010E948E1D03
:1051D0008090820290908302A0908402B090850219
:1051E000B70190E080E00E946A38A50194010E9416
:1051F000313A2DEC3CEC4CE45DE30E94CB38A50148
:1052000094010E94323A60938202709383028093E9
:105210008402909385020E94CF246091AD02709128
:10522000AE0290E080E00E946A386B017C01209120
:105230004D0730914E0740914F07509150070E9403
:1052400065388111B5C02091A1023091A202409130
:10525000A3025091A402C701B6010E94313A6B012A
:105260007C0120E030E0A9010E94463B18160CF0BA
:1052700095C020E030E040EA50E4C701B6010E944A
:10528000463B18160CF494C060919F027091A002E6
:1052900090E080E00E946A382091A1023091A20241
:1052A0004091A3025091A4020E94313A6B017C010B
:1052B00020E030E0A9010E94463B18160CF087C0A0
:1052C000C701B6010E94173B6530710508F083C025
:1052D00080914E01811105C080914D0181110E9484
:1052E000842081E080934E0110924D018091AD02A7
:1052F0009091AE02853F21E0920710F010920001DC
:1053000020910001211140C0843F9140E8F58FEFCA
:1053100090E00E948E1D0E948420C1E0C093000195
:105320000E94CD260E94FD27C093A5028EE00E9418
:105330002E20BC0190E080E00E946A3860938202D7
:105340007093830280938402909385021092970257
:1053500080919F029091A00224E630E030938D026C
:1053600020938C0220E233E030938B0220938A0258
:105370002AE030E03093890220938802880F991F39
:105380009093990280939802CF91FF90EF90DF90D5
:10539000CF90BF90AF909F908F90089520E030E025
:1053A00040EA50ECC701B6010E94653887FF6CCF18
:1053B0006091A1027091A2028091A3029091A40237
:1053C0000E94173B7093AE026093AD025DCFC701A0
:1053D000B601905877CF10924E0188CF0C9489393E
:1053E0002F923F924F925F926F927F928F929F92F5
:1053F000AF92BF92CF92DF92EF92FF920F931F93E3
:10540000CF93DF93CDB7DEB7E4970FB6F894DEBF46
:105410000FBECDBF1EA21DA218A61FA21AA619A6B6
:1054200050E040E060E772E0CE0185960E94AA2736
:1054300086E00E94FB1C21E0892B09F020E02093EC
:105440008702CE0101969AAB89AB0E940E1B96E0B3
:105450009093A707A1E0A093A6071092A50769A5BE
:105460007AA54DA15EA1FE01BB96FCABEBAB90E033
:1054700080E08617970730F4DA01A80FB91F4115AD
:10548000510521F410927302A3E7B2E02C9130E0B1
:105490002193319301968330910559F780919802B9
:1054A0009091990218A21F8E1AA219A21CA21BA2E7
:1054B0004AE0BE016F5F7F4F959587950E941B382C
:1054C000E9A9FAA901900020E9F73197AF0189A96C
:1054D0009AA9481B590BBE016F5F7F4FCE014F96B3
:1054E0000E94AA278DA19EA1009709F402C16F8D89
:1054F00078A16115710509F4FAC04FA158A52BA137
:105500003CA14217530708F4F2C00E94563D8BA1FC
:105510009CA19AA789A71CA21BA28F8D98A1009776
:1055200011F00E94023C5E0193E1A90EB11C84E0DF
:10553000282E312C912C812C89A59AA588169906A4
:1055400028F4EDA1FEA1309709F0E4C01092730297
:10555000E3E7F2E0ABA9BCA9CD90DD90BCABABAB6F
:10556000808190E08C199D09B2E3B89FB001B99F8A
:10557000700D1124072E000C880B990B0E946C38BB
:10558000F50120813181428153810E94323A2B0101
:105590003C0120E030E0A9010E9465388111BDC0C6
:1055A000D5014D925D926D927C92139701E022E3BA
:1055B00046E270E060E0C10104970E94461B0D2C9A
:1055C000000CEE08FF08F1E3CF1AD108E108F1085A
:1055D0000EEC1FEF20E030E040E850E4D5016D9183
:1055E0007D918D919C910E94323A2B013C01B80132
:1055F000012E000C880B990B0E946C389B01AC01AA
:10560000C301B2010E94323A0E94103B3092A207BD
:105610002092A1077093A4076093A307C701B60166
:105620000E94CB250E5C1F4FBFEFCB1ADB0AEB0AA3
:10563000FB0A0436110571F6EFEF8E1A9E0AF4E0AC
:10564000AF0EB11C2CE2220E311C83E088169104AF
:1056500009F072CF00E022E040E870E060E090E006
:1056600080E00E94461B2DE040E863E370E090E09C
:1056700080E00E94461B0E94651E0E94722086E008
:105680000E94FB1C892B09F0E0CE809187028111DA
:10569000DCCE0E948420EDA0FEA060E070E0CB0193
:1056A000E114F10419F0C7010E94F4378B01E114F1
:1056B000F10419F0C7010E94023CC801E4960FB63C
:1056C000F894DEBF0FBECDBFDF91CF911F910F9138
:1056D000FF90EF90DF90CF90BF90AF909F908F9012
:1056E0007F906F905F904F903F902F9008950E9411
:1056F000023C8F8D98A19EA38DA389A19AA198A702
:105700008FA38BA19CA19AA789A718A21F8E1AA26A
:1057100019A201CFE80DF91D1DCFC301B2019058A8
:105720002DEC3CEC4CE45FE30E94CB38A3019201EA
:105730000E94323AF501608371838283938336CF6E
:105740001F920F920FB60F9211242F933F934F93F6
:105750005F936F937F938F939F93AF93BF93EF93D9
:10576000FF9380EB96E00E94431CFF91EF91BF9165
:10577000AF919F918F917F916F915F914F913F91E9
:105780002F910F900FBE0F901F9018951F920F92A0
:105790000FB60F9211242F938F939F93EF93FF9344
:1057A000E091C006F091C1068081E091C606F091BB
:1057B000C70682FD1BC090818091C9068F5F8F73E1
:1057C0002091CA06821741F0E091C906F0E0E05549
:1057D000F94F958F8093C906FF91EF919F918F911B
:1057E0002F910F900FBE0F901F9018958081F4CFCE
:1057F0001F920F920FB60F9211242F933F938F9306
:105800009F93AF93BF938091750290917602A09180
:105810007702B09178023091740223E0230F2D3784
:1058200058F50196A11DB11D209374028093750255
:1058300090937602A0937702B093780280917902D8
:1058400090917A02A0917B02B0917C020196A11DF9
:10585000B11D8093790290937A02A0937B02B0935A
:105860007C02BF91AF919F918F913F912F910F90AB
:105870000FBE0F901F90189526E8230F0296A11DCA
:10588000B11DD2CF1F920F920FB60F9211242F93FA
:105890003F934F935F936F937F938F939F93EF9378
:1058A000FF9383B1817029B190917F02981709F419
:1058B0009DC030E0220F232F221F330B922F8093A5
:1058C0007F0240917E02241709F490C020937E024B
:1058D0002091880230918902981719F0319521950D
:1058E0003109409198025091990260918C02709117
:1058F0008D02240F351F261737070CF48BC020911B
:10590000880230918902981719F031952195310953
:10591000409198025091990260918A0270918B0295
:10592000240F351F621773070CF46FC04091880273
:1059300050918902981719F051954195510920917C
:10594000980230919902240F351F309399022093C9
:10595000980241E0981340E020917D02421709F43B
:1059600040C02091880230918902981719F0319532
:10597000219531096091980270919902E0918C0211
:10598000F0918D02260F371F2E173F070CF44CC0E5
:105990002091880230918902981719F0319521954C
:1059A00031096091980270919902E0918A02F09118
:1059B0008B02260F371FE217F3078CF12091880224
:1059C00030918902981719F031952195310980910C
:1059D000980290919902820F931F9093990280935D
:1059E000980240937D0281E08093A502FF91EF91A0
:1059F0009F918F917F916F915F914F913F912F91E7
:105A00000F900FBE0F901F90189520918A02309131
:105A10008B029BCF20918C0230918D0296CF80918A
:105A20008A0290918B02D9CF80918C0290918D0245
:105A3000D4CF18950F931F93CF93DF93E0EBF6E04D
:105A40001382128288EE93E0A0E0B0E08483958315
:105A5000A683B78388E492E09183808385EC90E00D
:105A60009587848784EC90E09787868780EC90E028
:105A7000918B808B81EC90E0938B828B82EC90E019
:105A8000958B848B86EC90E0978B868B118E128E93
:105A9000138E148EE5E9F7E01382128216821782C4
:105AA00080E180871582148212868AE592E09183D4
:105AB0008083158614861786168681E0808B118A6E
:105AC000828B138AC9E5D7E021E537E03F8F2E8F1F
:105AD00025E537E03D8F2C8F2DE437E039A328A34F
:105AE0001AAE1AAA1BAA1CAA1DAA40E050E06FE732
:105AF00073E44EAB5FAB68AF79AF44E650E060E073
:105B000070E04EA75FA768AB79AB21E030E0398F3A
:105B1000288F3B8F2A8F8BAF80E090E0A0E3B1E429
:105B200088839983AA83BB8380E090E0A0E0BFE3F1
:105B30008C839D83AE83BF8380E090E0A0E8BFE3C9
:105B400088879987AA87BB8780E090E0A0E3B1ECC3
:105B50008C879D87AE87BF878DEC9CECACE4BDEB5A
:105B6000888B998BAA8BBB8B80E090E0A0E2B1EC94
:105B70008C8B9D8BAE8BBF8B0E943D1E0EA51FA5EF
:105B800028A939A9601B710B820B930B6AA37BA315
:105B90008CA39DA3DF91CF911F910F910895CF9377
:105BA000DF93CDB7DEB72A970FB6F894DEBF0FBEEE
:105BB000CDBF789484B5826084BD84B5816084BD96
:105BC00085B5826085BD85B5816085BD80916E009B
:105BD000816080936E0010928100809181008260CC
:105BE0008093810080918100816080938100809109
:105BF00080008160809380008091B10084608093F8
:105C0000B1008091B00081608093B00080917A00F3
:105C1000846080937A0080917A00826080937A0019
:105C200080917A00816080937A0080917A00806808
:105C300080937A001092C1001092B90088E480939A
:105C4000B8000E945B1E80E00E94511E03EC1FE220
:105C500042EEE42E4FE2F42EF80184910E94511E90
:105C60000F5F1F4FE016F106B9F70E94491E11E0C1
:105C70001093B8000E94651E82E480939D0760E047
:105C80008EE00E94521D60E08FE00E94521D61E094
:105C900085E00E94521D61E089E00E94521D62E091
:105CA00087E00E94521D62E088E00E94521D62E07F
:105CB00086E00E94521D62E08AE00E94521D8FEF32
:105CC00090E00E948E1D60E085E00E94241D80917E
:105CD0007A00876080937A0080917A008860809350
:105CE0007A00789410936B00109368001BBB90E0CF
:105CF00080E00E94EE29182F81E090E00E94EE29BA
:105D0000912F8F30984009F0B5C082E090E00E945A
:105D1000EE29182F83E090E00E94EE29912F9093B6
:105D200047018093460184E090E00E94EE29182FFD
:105D300085E090E00E94EE29912F90934501809399
:105D4000440186E090E00E94EE298093430187E0C1
:105D500090E00E94EE2980934C0188E090E00E9440
:105D6000EE2980934B0189E090E00E94EE29809318
:105D70004A018AE090E00E94EE298093AF028BE016
:105D800090E00E94EE2991E0811101C090E0909393
:105D900049018CE090E00E94EE2991E0811101C060
:105DA00090E0909348018DE090E00E94EE2980936E
:105DB000AC028EE090E00E94EE29282E80934201F2
:105DC0008FE090E00E94EE298093A80280E190E0AD
:105DD0000E94EE2991E0811101C090E0909386022B
:105DE00092E0892E91E0992E2FE4A22E21E0B22E8E
:105DF00031E1E32EF12C312C231409F447C010E0DB
:105E000000E0C701800F911F0E94EE29F501E00F0D
:105E1000F11F80830F5F1F4F0630110591F7670157
:105E200026E0C20ED11C3EE0E30EF11C3401C60197
:105E30000E94EE29082F10E0102F0027F301118394
:105E400000832601F2E04F0E511CC60101960E940C
:105E5000EE29082BF301019311933F0162014E14C7
:105E60005F0429F73394F8E08F0E911C26E0A20E10
:105E7000B11CC2CF68E090E080E00E94E9276FE0AB
:105E800081E090E00E94E9270E94FD2710918602A0
:105E900080EC111101C088EC0E94821E80EA111171
:105EA00001C081EA0E94821E0E94B41F9093810269
:105EB000809380020E945C209093A7028093A602A8
:105EC00000914601109147011093A00200939F0298
:105ED0008EE00E942E20BC0190E080E00E946A3893
:105EE0006093820270938302809384029093850270
:105EF0000E94F01F0E94CF2420E030E040EA51E4ED
:105F00006091A1027091A2028091A3029091A402DB
:105F10000E94323A6B017C01B80190E080E00E945F
:105F20006A389B01AC01C701B6010E94653887FF42
:105F300004C090E080E00E948E1D10928B071092AA
:105F40008C0710928D0710928E07412C512CBFE7C1
:105F50006B2EB3E47B2E40928F0750929007609295
:105F6000910770929207A0907707B0907807809180
:105F70009307F501C080D180E280F380882311F47B
:105F80000C94C837A3019201C701B6010E94463B99
:105F9000181634F5F5014082518262827382809036
:105FA0007F0790908007A0908107B0908207C090F3
:105FB0008F07D0909007E0909107F0909207A7018B
:105FC0009601C501B4010E94463B1816C4F4C09264
:105FD0007F07D0928007E0928107F09282071FC06E
:105FE00020E030E0A901C701B6010E94653887FFB3
:105FF000D6CFF5011082118212821382D0CFC090C9
:106000008B07D0908C07E0908D07F0908E07A7014A
:106010009601C501B4010E94653887FDD8CF81E0A3
:106020008093930783B1817080937F0289B190E060
:10603000880F892F881F990B80937E0220917F0201
:1060400090917E0281E0291380E080937D0284E6B6
:1060500090E090938D0280938C0280E293E0909385
:106060008B0280938A028AE090E090938902809369
:106070008802000F111F10939902009398020E944A
:106080003D1E60939B0270939C0280939D029093AF
:106090009E020E9484200E948420209098023090CA
:1060A00099029101359527953A8729873093A00267
:1060B00020939F0286E00E94FB1C482E81119EC007
:1060C00080919702882309F499C00E9484200E943D
:1060D0003D1E6B017C01C0929302D0929402E0922B
:1060E0009502F092960286E00E94FB1C892B59F4DF
:1060F0000E943D1E6C197D098E099F09643F714005
:106100008105910580F30E943D1E6C197D098E0961
:106110009F09643F71408105910508F43EC48FEFEB
:1061200090E00E948E1D0E948420512C7AE0672E00
:10613000712C10928E02852D0E949121582EF7E02D
:10614000F81708F438C0E82FF0E0E755FF4C0C943E
:10615000603BC3306933E033463454348E349C346E
:10616000A63420E030E0A901C701B6010E946538DD
:1061700087FF55CF10927F071092800710928107FA
:10618000109282074CCF6EE1662E712C81E08093D5
:106190008E02852D0E949121582E22E0821709F44B
:1061A00034C2281708F4E8C0882309F410C131E08C
:1061B000831709F40FC10E94FD2781E08093A50297
:1061C00029853A853093A00220939F0284E690E0CF
:1061D00090938D0280938C0280E293E090938B02E7
:1061E00080938A028AE090E09093890280938802EB
:1061F000C1018E7F909399028093980240929702FA
:106200008091A902882309F110914A011123E9F034
:106210000E943D1EC0908F02D0909002E0909102AB
:10622000F09092026C197D098E099F0928EE33E0E7
:1062300040E050E00E94003A211738F01092A90285
:106240000E94842081E080934D018091A5028823E3
:10625000E9F18091AA02882349F120E030E040EA88
:1062600051E46091A1027091A2028091A3029091E9
:10627000A4020E94323A6B017C0160919F027091EE
:10628000A00290E080E00E946A389B01AC01C70147
:10629000B6010E94653887FF04C090E080E00E944C
:1062A0008E1D0E94842081E080934D011092A502F2
:1062B0001092AA021092AB020E943D1E60939B02B4
:1062C00070939C0280939D0290939E020E943D1EBB
:1062D00000919B0210919C0220919D0230919E02A0
:1062E000601B710B820B930B20E63AEE40E050E00E
:1062F0000E94003A122F20939A028091AA028111E3
:106300000BC080914C01882339F0281728F081E0D8
:106310008093AA020E9484208091AB0281110BC05D
:1063200080914B01882339F0181728F081E0809381
:10633000AB020E9484200E94AC280E94A2220E94EC
:106340003D1E80919E07362F381B832F90919F070B
:10635000992309F438C33093A00710929F0780E077
:1063600090E0892B09F499CE0E942F1C882309F410
:1063700094CE0E94000091CE83E0581609F448C1E3
:1063800094E0591218CF80914201883008F0FECE77
:1063900091E0980F909342018093AC020E94A2205A
:1063A000E091AC0228E0E29FF0011124EE5FFE4F85
:1063B00088ED90E09183808324E331E0338322836E
:1063C00086E891E09583848377826682DFCE0E949F
:1063D000CD26DCCE8E010F5F1F4F812C912C5401F6
:1063E000839448EEE42E43E0F42ECC24C394D12CC5
:1063F000E091AC0224E0E29FF0011124C401019776
:10640000E80FF91FEE0FFF1FEE5FFE4F80819181B5
:106410009093A00280939F02E8ECF0E0F0938D024D
:10642000E0938C02F0928B02E0928A02D092890271
:10643000C0928802880F991F9093990280939802C6
:10644000F1E0F0934D0186E00E94FB1C21E0892BD6
:1064500009F020E0209387020E940E1B22E0209387
:10646000A7070E94AC280E94A2221092A2071092B5
:10647000A1071092A4071092A30788E090E30E945E
:10648000961FC501B4010E94CB258EE692E00E94C2
:106490007A2580914E011092A2071092A1078823BD
:1064A00009F48BC080E190E09093A4078093A30748
:1064B0008BEF9FE20E94961F1092A2071092A107F5
:1064C000E0E2F0E0F093A407E093A30784EF9FE2FB
:1064D0000E94961F60919802709199027595679538
:1064E000072E000C880B990B0E94CB250E9472206E
:1064F0000E94651E86E00E94FB1C892B09F0ACCF30
:10650000809187028111A8CF809198029091990281
:1065100095958795F801819391938F010E9484202E
:106520006AE070E080E090E00E940B1EFFEF8F1A9F
:106530009F0AAF0ABF0A24E082169104A104B104A5
:1065400009F056CF8FEF90E00E948E1D8BEA94E009
:106550000197F1F70E94F01F0E94173B4B017887CB
:106560006F83C980DA800B811C81C6014E9680172B
:10657000910708F00BCEED80FE80C8014E968E1577
:106580009F0508F003CE87E080938E0280E00E9492
:106590009121882309F4FACDE091AC0238E0E39F21
:1065A000F0011124EE5FFE4FD182C082138302837B
:1065B000F582E48297828682E9CD20E130E0309353
:1065C000A4072093A3078EEE9FE20E94961F60917E
:1065D00082027091830280918402909185020E94D0
:1065E000173B90E080E04AE00E9487251092A207C6
:1065F0001092A10780E290E09093A4078093A307F4
:1066000082EE9FE20E94961F71CF0E94A220BECD13
:1066100087E080938E0210914201113009F4B6CDCB
:1066200080E00E949121882309F4B0CD0091AC0252
:10663000812F8150990BBC010817190639F40150BC
:106640000093AC02115010934201A0CD802F90E036
:1066500086179707BCF7E6E00E9FD001112450E0A3
:1066600040E09C012F5F3F4FFA01EA0FFB1FE15B07
:10667000FE4FF680F0824F5F5F4F46305105A1F725
:10668000E3E0220F331FEA95E1F7F901EE5FFE4FD9
:1066900020813181A3E0880F991FAA95E1F7DC01E1
:1066A000AE5FBE4F11963C932E93828193811396D9
:1066B0009C938E9312978481958115969C938E93CB
:1066C00014978681978117969C938E9316970F5FE8
:1066D000BDCF82E080938E0210E040E9C42EDD241D
:1066E000D39454E6A52EB12C60E2862E63E0962E5C
:1066F00074E1E72EF12C812F0E949121182F813017
:1067000021F130F0823009F43FC00E94FD2711CD05
:106710008091460190914701B0928D02A0928C0227
:1067200090928B0280928A02709289026092880213
:10673000880F991F90939902809398020E94F029E4
:106740009093470180934601D6CF80914401909168
:106750004501E8E2F0E0F0938D02E0938C02D092E4
:106760008B02C0928A027092890260928802880F1E
:10677000991F90939902809398020E94F029909318
:10678000450180934401B7CF8091430190E0F0929E
:106790008D02E0928C0228EC30E030938B02209343
:1067A0008A027092890260928802880F991F9093E2
:1067B0009902809398020E94F029809343019BCF15
:1067C00083E080938E0210E0812F0E949121182F88
:1067D0008130F1F1F8F0823009F097CF80914A01D1
:1067E00090E010928D0210928C02E8E6F1E0F093B6
:1067F0008B02E0938A027092890260928802880F6D
:10680000991F90939902809398020E94F029809397
:106810004A01DACF80914C0190E010928D021092E3
:106820008C02ECE3F0E0F0938B02E0938A0221E02B
:1068300030E03093890220938802880F991F90934B
:106840009902809398020E94F02980934C01BCCF5A
:1068500080914B0190E010928D0210928C02E8E73B
:10686000F0E0F0938B02E0938A0225E030E0309371
:10687000890220938802880F991F90939902809330
:1068800098020E94F02980934B019ECF84E0809370
:106890008E02809149010E94912191E0811101C0F5
:1068A00090E09093490145CC10E06AE0E62E75E057
:1068B000D72EE9E0CE2EE0928E02812F0E94912108
:1068C000182F882321F08130E1F000E009C0D09238
:1068D0008E028091AF020E9491218093AF0201E06D
:1068E000F090860280ECF11001C088EC0E94821EBC
:1068F00080EAF11001C081EA0E94821E0111DBCF03
:1069000004CF80918602C0928E020E94912191E074
:10691000811101C090E090938602E1CF86E08093E0
:106920008E02809148010E94912191E0811101C065
:1069300090E090934801FDCB88E080938E02809197
:10694000A8020E9491218093A802F3CB86E00E94C6
:10695000FB1C21E0892B09F020E0209387020E9494
:106960000E1BEE24E39400E420E44FE050E370E0DB
:1069700060E080E290E00E948C1A0E94651E0E94F6
:10698000722086E00E94FB1C892BC9F78091870248
:106990008111F5CF0E948420CCCB8091A90291E097
:1069A00089278093A902882351F00E943D1E60939D
:1069B0008F0270939002809391029093920281E0F3
:1069C0008093A5021BCC90919D07391748F48F5FE7
:1069D000891708F0C4CC81E083BF889513BEBFCC73
:1069E00011E010939F0760939E0780919907909103
:1069F0009A07019690939A07809399078091AF0226
:106A0000882309F4A1C20E940E1B01E020E440E8A3
:106A100070E060E090E080E00E94461B1093A707C2
:106A20001093A6071092A507E12C00E120E14EE8A3
:106A300052E370E060E090E080E00E948C1A83E115
:106A400090E09093A2078093A10784E090E0909358
:106A5000A4078093A3078091AC02E6E08E9FC0015B
:106A60001124815B9E4F0E947A258091AD02909106
:106A7000AE02853F914008F032C28091AB02811195
:106A800030C28091AA0281112EC28091A902811187
:106A90002CC280914E0181112AC220E030E044E3F3
:106AA00053E4609151077091520780915307909180
:106AB00054070E94653887FF1CC285E025E330E05B
:106AC0003093A2072093A10721E030E03093A40780
:106AD0002093A30792E09093A707C82ED12C909102
:106AE000A802CC0CDD1C911106C2F601EA5CFD4F38
:106AF00040815181E12C0EE02CE161E070E080E505
:106B000090E00E948C1AF601E85DFD4F40815181B2
:106B1000E12C00E120E170E060E080E790E00E947D
:106B20008C1A81E08093A70720E148E452E360E1FA
:106B300070E090E080E00E948C1A20E148E252E38D
:106B400060E270E090E080E00E948C1A03E110E0C7
:106B50001093A2070093A10720E130E03093A4072F
:106B60002093A3070E94F01F41E00E94F52588EFC3
:106B70000E94911F86E292E30E94961F1093A20743
:106B80000093A10788E190E09093A4078093A30766
:106B90000E94B41FBC0190E080E00E946A3820E0AF
:106BA00030E04AE754E40E949E3A42E00E94F52514
:106BB00084E292E30E94961F1093A2070093A1071C
:106BC00080E290E09093A4078093A3076091A602CF
:106BD0007091A70290E080E00E946A3820E030E0E7
:106BE0004AE754E40E949E3A41E00E94F52582E281
:106BF00092E30E94961F1093A2070093A10788E2D8
:106C000090E09093A4078093A3078BE192E30E9406
:106C1000961F89E390E09093A2078093A10782E1F9
:106C200090E09093A4078093A30784E08093A70744
:106C30006091AD027091AE02653F91E0790708F472
:106C40007DC187E192E30E94961F20E248E460E163
:106C500070E087E390E00E94971B81E08093A70794
:106C60002EE046E661E370E081E090E00E94971B31
:106C70002091AD023091AE02253FE1E03E07C0F425
:106C8000A4E6B0E00E94223A24EF31E040E050E078
:106C90000E949F39BA01A9014E5F5F4F6F4F7F4F2E
:106CA00000E02EE061E370E081E090E00E94461B8E
:106CB00060914D0770914E0780914F07909150075A
:106CC0000E94103B9B01AC01A4E6B0E00E94BE39DB
:106CD00034EFC32EDD24D394E12CF12CA7019601CF
:106CE0000E949F39DA01C9010296A11DB11D0297C8
:106CF00000E02DE043E062E370E00E94461B6091FB
:106D00004D0770914E0780914F07909150070E9458
:106D1000103B9B01AC01A4E6B0E00E94BE39A70184
:106D200096010E949F39DA01C9010296A11DB11D89
:106D3000039724E045E06CE370E00E94461B6091FD
:106D40004D0770914E0780914F07909150070E9418
:106D5000103B9B01AC01A4E6B0E00E94BE39A70144
:106D600096010E949F3989019A010E5F1F4F2F4F94
:106D70003F4F0150110941E3E42EF12C41E0B701EE
:106D8000C8010E946E1AFFEFEF1AFF0A2DE3E21608
:106D9000F104A1F760914D0770914E0780914F0764
:106DA000909150070E94103B9B01AC01A4E6B0E01B
:106DB0000E94BE3924EF31E040E050E00E949F394C
:106DC000DA01C9010296A11DB11D0397EE24E394D7
:106DD00004E025E043E152E36BE370E00E948C1A8B
:106DE0002EE047E161E370E088E690E00E94971BA7
:106DF0006091510770915207809153079091540709
:106E00000E94103B9B01AC012F5F310941095109E0
:106E1000A7E1B0E00E94BE39CC24C394DD24DA940B
:106E2000ED2CFD2CA70196010E949F39422F00E016
:106E30002EE061E370E088E690E00E94461B10922D
:106E4000A60781E08093A50782E090E09093A207D7
:106E50008093A10707E310E01093A4070093A30712
:106E600060914D0770914E0780914F0790915007A8
:106E700040E00E94F52588EF0E94911F81E192E396
:106E80000E94961F89E690E09093A2078093A10745
:106E90001093A4070093A3076091510770915207C4
:106EA00080915307909154070E94103B9B01AC01C5
:106EB0002F5F310941095109A4E6B0E00E94BE39B3
:106EC000A70196010E949F39CA01B9010E94CB25F2
:106ED0008FE092E30E94961F0E94651E40CA80E0E8
:106EE000EDCD81E0EBCD82E0E9CD83E0E7CD84E03C
:106EF000E5CD86E0E3CD8330C1F038F4813069F030
:106F0000823081F088E692E30AC08530A1F080F0FB
:106F10008630C1F78EE692E302C08AE892E30E94CF
:106F2000961FF1CD84E892E3FACF8EE792E3F7CF94
:106F300088E792E3F4CF83E792E3F1CF90E080E03B
:106F40004AE00E94872581CE0E940E1B1092A60760
:106F50001093A50787E08093A7071092A2071092CD
:106F6000A10788E090E09093A4078093A307609125
:106F7000AD027091AE02653F31E0730718F08EEA02
:106F800092E3A8CF90E080E04AE00E948725A4CF5A
:106F9000C0927F07D0928007E0928107F09282072B
:106FA000E0917507F091760780819181A281B3818C
:106FB0008093830790938407A0938507B0938607F7
:106FC00020E030E04FE753E4C701B6010E94463BA2
:106FD00018160CF0C6C840927F0750928007609246
:106FE0008107709282071BC81F93FC01992788278D
:106FF000BC01E89411911032E9F3193010F01E3001
:10700000C8F31B3251F01D3249F4689406C00E9447
:107010002638610F711D811D911D119110531A3079
:10702000B0F33EF490958095709561957F4F8F4FAA
:107030009F4F1F910895BB274A3031F4992322F4C2
:10704000BDE2909581959F4F0C943C38592F482F65
:10705000372F262F660F771F881F991F660F771F00
:10706000881F991F620F731F841F951F660F771F5C
:10707000881F991F0895BB27FB015527AA27880F52
:10708000991FAA1FA41710F0A41B83955051B9F79C
:10709000A05DAA3308F0A95DA193009779F7B1111B
:1070A000B1931192CB010C945538DC01FC01672F90
:1070B00071917723E1F7329704C07C916D937083CF
:1070C0006291AE17BF07C8F308950E94A73808F46D
:1070D00081E00895E89409C097FB3EF4909580956F
:1070E000709561957F4F8F4F9F4F9923A9F0F92F8E
:1070F00096E9BB279395F695879577956795B7950C
:10710000F111F8CFFAF4BB0F11F460FF1BC06F5FF1
:107110007F4F8F4F9F4F16C0882311F096E911C003
:10712000772321F09EE8872F762F05C0662371F024
:1071300096E8862F70E060E02AF09A95660F771F38
:10714000881FDAF7880F9695879597F90895990F14
:107150000008550FAA0BE0E8FEEF16161706E80721
:10716000F907C0F012161306E407F50798F0621B42
:10717000730B840B950B39F40A2661F0232B242B17
:10718000252B21F408950A2609F4A140A6958FEF36
:10719000811D811D08950E94DE380C944F390E9494
:1071A000413938F00E94483920F0952311F00C94B1
:1071B00038390C943E3911240C9483390E9460397B
:1071C00070F3959FC1F3950F50E0551F629FF0013A
:1071D000729FBB27F00DB11D639FAA27F00DB11D53
:1071E000AA1F649F6627B00DA11D661F829F2227DC
:1071F000B00DA11D621F739FB00DA11D621F839F63
:10720000A00D611D221F749F3327A00D611D231F38
:10721000849F600D211D822F762F6A2F11249F5786
:1072200050409AF0F1F088234AF0EE0FFF1FBB1F89
:10723000661F771F881F91505040A9F79E3F510548
:1072400080F00C9438390C9483395F3FE4F3983E16
:10725000D4F3869577956795B795F795E7959F5FF2
:10726000C1F7FE2B880F911D9695879597F9089584
:1072700097F99F6780E870E060E008959FEF80ECE9
:10728000089500240A94161617061806090608958C
:1072900000240A9412161306140605060895092EF2
:1072A0000394000C11F4882352F0BB0F40F4BF2B61
:1072B00011F460FF04C06F5F7F4F8F4F9F4F0895A1
:1072C00057FD9058440F551F59F05F3F71F0479597
:1072D000880F97FB991F61F09F3F79F0879508957C
:1072E000121613061406551FF2CF4695F1DF08C09B
:1072F000161617061806991FF1CF869571056105B8
:1073000008940895E894BB2766277727CB0197F95F
:107310000895F999FECF92BD81BDF89A992780B55D
:107320000895262FF999FECF1FBA92BD81BD20BDC9
:107330000FB6F894FA9AF99A0FBE01960895052EA1
:1073400097FB1EF400940E94B63957FD07D00E94A7
:10735000003A07FC03D04EF40C94B6395095409592
:10736000309521953F4F4F4F5F4F089590958095F1
:10737000709561957F4F8F4F9F4F08950E94223ADD
:10738000A59F900DB49F900DA49F800D911D112479
:1073900008952F923F924F925F926F927F928F92B9
:1073A0009F92AF92BF92CF92DF92EF92FF920F9394
:1073B0001F93CF93DF93CDB7DEB7CA1BDB0B0FB69E
:1073C000F894DEBF0FBECDBF09942A88398848885B
:1073D0005F846E847D848C849B84AA84B984C884F1
:1073E000DF80EE80FD800C811B81AA81B981CE0FE8
:1073F000D11D0FB6F894DEBF0FBECDBFED010895CD
:10740000A1E21A2EAA1BBB1BFD010DC0AA1FBB1FA8
:10741000EE1FFF1FA217B307E407F50720F0A21B1A
:10742000B30BE40BF50B661F771F881F991F1A9487
:1074300069F760957095809590959B01AC01BD01B1
:10744000CF010895A29FB001B39FC001A39F700D0B
:10745000811D1124911DB29F700D811D1124911D5C
:1074600008955058BB27AA270E94493A0C944F39D7
:107470000E94413938F00E94483920F039F49F3F8A
:1074800019F426F40C943E390EF4E095E7FB0C94C5
:107490003839E92F0E94603958F3BA176207730729
:1074A0008407950720F079F4A6F50C9482390EF440
:1074B000E0950B2EBA2FA02D0B01B90190010C0104
:1074C000CA01A0011124FF27591B99F0593F50F41C
:1074D000503E68F11A16F040A22F232F342F442774
:1074E000585FF3CF469537952795A795F04053956C
:1074F000C9F77EF41F16BA0B620B730B840BBAF03C
:107500009150A1F0FF0FBB1F661F771F881FC2F7A6
:107510000EC0BA0F621F731F841F48F487957795BA
:107520006795B795F7959E3F08F0B0CF9395880F74
:1075300008F09927EE0F9795879508950E94B23A23
:107540000C944F390E94483958F00E94413940F05C
:1075500029F45F3F29F00C94383951110C94833988
:107560000C943E390E94603968F39923B1F3552396
:1075700091F3951B550BBB27AA2762177307840746
:1075800038F09F5F5F4F220F331F441FAA1FA9F3DC
:1075900035D00E2E3AF0E0E832D091505040E695CA
:1075A000001CCAF72BD0FE2F29D0660F771F881F2B
:1075B000BB1F261737074807AB07B0E809F0BB0B1E
:1075C000802DBF01FF2793585F4F3AF09E3F510532
:1075D00078F00C9438390C9483395F3FE4F3983E8B
:1075E000D4F3869577956795B795F7959F5FC9F71B
:1075F000880F911D9695879597F90895E1E0660F9C
:10760000771F881FBB1F621773078407BA0720F014
:10761000621B730B840BBA0BEE1F88F7E09508957D
:107620000E94173B6894B1110C94833908950E940D
:10763000683988F09F5798F0B92F9927B751B0F063
:10764000E1F0660F771F881F991F1AF0BA95C9F7E6
:1076500014C0B13091F00E948239B1E008950C94C9
:107660008239672F782F8827B85F39F0B93FCCF37C
:10767000869577956795B395D9F73EF49095809563
:10768000709561957F4F8F4F9F4F08950E94A73847
:1076900008F48FEF08950E94A738880B990B08957E
:1076A000DB018F939F930E94BE39BF91AF91A29F40
:1076B000800D911DA39F900DB29F900D11240895F0
:1076C000EE0FFF1F0590F491E02D09940F931F9387
:1076D000CF93DF938230910510F482E090E0E09147
:1076E000AB07F091AC0730E020E0B0E0A0E03097CD
:1076F00099F42115310509F44AC0281B390B2430AF
:107700003105D8F58A819B816115710589F1FB01ED
:1077100093838283FE0111C04081518102811381D4
:1077200048175907E0F04817590799F4109761F086
:1077300012960C93129713961C933296CF01DF91F9
:10774000CF911F910F9108950093AB071093AC0751
:10775000F4CF2115310551F04217530738F0A90134
:10776000DB019A01BD01DF01F801C1CFEF01F9CFC3
:107770009093AC078093AB07CDCFFE01E20FF31FD0
:10778000819391932250310939832883D7CF209157
:10779000A9073091AA07232B41F420918101309150
:1077A00082013093AA072093A90720917F0130918D
:1077B00080012115310541F42DB73EB74091830179
:1077C00050918401241B350BE091A907F091AA0781
:1077D000E217F307A0F42E1B3F0B2817390778F0A8
:1077E000AC014E5F5F4F2417350748F04E0F5F1F07
:1077F0005093AA074093A907819391939FCFF0E0FC
:10780000E0E09CCFCF93DF930097E9F0FC01329743
:1078100013821282A091AB07B091AC07ED0130E06A
:1078200020E01097A1F420813181820F931F2091D5
:10783000A9073091AA072817390709F061C0F0930A
:10784000AA07E093A907DF91CF910895EA01CE1727
:10785000DF07E8F54A815B819E0141155105B1F7CB
:10786000E901FB83EA8349915991C40FD51FEC17B5
:10787000FD0761F4808191810296840F951FE901D3
:1078800099838883828193819B838A83F0E0E0E0FF
:1078900012968D919C9113970097B9F52D913C917B
:1078A0001197CD010296820F931F2091A907309165
:1078B000AA072817390739F6309751F51092AC0707
:1078C0001092AB07B093AA07A093A907BCCFD383AC
:1078D000C28340815181840F951FC817D90761F475
:1078E0004E5F5F4F88819981480F591F51834083B4
:1078F0008A819B81938382832115310509F0B0CF62
:10790000F093AC07E093AB079ECFFD01DC01C0CF45
:1079100013821282D7CFB0E0A0E0E1E9FCE30C943F
:10792000CB398C01009751F4CB010E94663B8C014E
:10793000C801CDB7DEB7E0E10C94E739FC01E60FF2
:10794000F71F9C0122503109E217F30708F49DC08C
:10795000D901CD91DC911197C617D70798F0C530A2
:10796000D10530F3CE0104978617970708F3C61B9D
:10797000D70B2297C193D1936D937C93CF010E9433
:10798000023CD6CF5B01AC1ABD0A4C018C0E9D1E89
:10799000A091AB07B091AC07512C412CF12CE12CFC
:1079A000109731F58091A9079091AA07881599053C
:1079B00009F05CC04616570608F058C080917F0158
:1079C00090918001009741F48DB79EB7409183015B
:1079D00050918401841B950BE817F90708F055C0F6
:1079E000F093AA07E093A907F90171836083A0CF00
:1079F0008D919C91119712966C90129713967C9092
:107A00001397A815B90559F56C0142E0C40ED11CB5
:107A1000CA14DB0420F1AC014A195B09DA011296A1
:107A2000159780F06282738251834083D9016D93F0
:107A30007C93E114F10471F0D7011396FC93EE935B
:107A4000129776CF22968C0F9D1FF9019183808328
:107A5000F301EFCFF093AC07E093AB0769CF481683
:107A6000590608F42C017D01D3019ACFCB010E9465
:107A7000663B7C01009749F0AE01B8010E944D3D84
:107A8000C8010E94023C870153CF10E000E050CFB4
:107A900081E090E0F8940C945D3DFB01DC0102C0B4
:107AA00001900D9241505040D8F70895FB01DC0140
:107AB00001900D920020E1F70895F894FFCF01FFA7
:107AC000D800340186011E00000000000000000004
:107AD00000000000000000000000000000000000A6
:107AE0000000000000000000000000000000000096
:107AF0000000000000000000000000000000000086
:107B0000013C960040010101280F0501014243316B
:107B10002E35000000000000000000000000000002
:107B20000000000000000000000000000000000055
:107B3000000000000000000000000000000000AD98
:107B400007800078092809D80888083808E80798C5
:107B5000074807F8067809A80658060806B8056811
:107B6000051805C80478046805C804280478046862
:107B700005D80388033803E80298024802F801A8F0
:107B80000158010801F801A801B80068006805085B
:107B900027E825C824A823882268214820281F0810
:107BA0001EE81CC81B0827A81A8819681808274847
:107BB00017281668184817081528166818E813C8F3
:107BC00012A8118810680F6821480E280D080CE8CB
:107BD0000A480E280DA811C80968180906040402ED
:107BE000020202020203C828A8288828283268282E
:107BF00048282828382A002AC829902958292029C5
:107C0000E82800000000651CC51BF21BB21C231CE9
:107C1000011C151C000000008F1EC51BB11FC41BDA
:107C20006E616E00696E66006F7666002F3300002D
:107E0000112484B714BE81FFF0D085E080938100F7
:107E100082E08093C00088E18093C10086E0809377
:107E2000C20080E18093C4008EE0C9D0259A86E02C
:107E300020E33CEF91E0309385002093840096BBD3
:107E4000B09BFECF1D9AA8958150A9F7CC24DD24C4
:107E500088248394B5E0AB2EA1E19A2EF3E0BF2EE7
:107E6000A2D0813461F49FD0082FAFD0023811F036
:107E7000013811F484E001C083E08DD089C08234E0
:107E800011F484E103C0853419F485E0A6D080C0E4
:107E9000853579F488D0E82EFF2485D0082F10E0AE
:107EA000102F00270E291F29000F111F8ED06801E7
:107EB0006FC0863521F484E090D080E0DECF843638
:107EC00009F040C070D06FD0082F6DD080E0C81688
:107ED00080E7D80618F4F601B7BEE895C0E0D1E017
:107EE00062D089930C17E1F7F0E0CF16F0E7DF06D8
:107EF00018F0F601B7BEE89568D007B600FCFDCFD4
:107F0000A601A0E0B1E02C9130E011968C91119780
:107F100090E0982F8827822B932B1296FA010C0160
:107F200087BEE89511244E5F5F4FF1E0A038BF0790
:107F300051F7F601A7BEE89507B600FCFDCF97BE46
:107F4000E89526C08437B1F42ED02DD0F82E2BD052
:107F50003CD0F601EF2C8F010F5F1F4F84911BD097
:107F6000EA94F801C1F70894C11CD11CFA94CF0C13
:107F7000D11C0EC0853739F428D08EE10CD085E9AC
:107F80000AD08FE07ACF813511F488E018D01DD067
:107F900080E101D065CF982F8091C00085FFFCCF94
:107FA0009093C60008958091C00087FFFCCF809118
:107FB000C00084FD01C0A8958091C6000895E0E648
:107FC000F0E098E1908380830895EDDF803219F02E
:107FD00088E0F5DFFFCF84E1DECF1F93182FE3DFCA
:107FE0001150E9F7F2DF1F91089580E0E8DFEE27F6
:047FF000FF270994CA
:027FFE00040479
:00000001FF
